 classfloadhk007

 Timestamp is 68b05017 (reproducible build file hash)

 Preferred load address is 0000000180000000

 Start         Length     Name                   Class
 0001:00000000 00004800H .text$mn                CODE
 0001:00004800 00000036H .text$mn$00             CODE
 0001:00004836 00000092H .text$x                 CODE
 0002:00000000 000001d8H .idata$5                DATA
 0002:000001d8 00000038H .00cfg                  DATA
 0002:00000210 00000008H .CRT$XCA                DATA
 0002:00000218 00000008H .CRT$XCZ                DATA
 0002:00000220 00000008H .CRT$XIA                DATA
 0002:00000228 00000008H .CRT$XIC                DATA
 0002:00000230 00000008H .CRT$XIZ                DATA
 0002:00000238 00000008H .CRT$XLA                DATA
 0002:00000240 00000008H .CRT$XLZ                DATA
 0002:00000248 00000008H .CRT$XPA                DATA
 0002:00000250 00000008H .CRT$XPZ                DATA
 0002:00000258 00000008H .CRT$XTA                DATA
 0002:00000260 00000010H .CRT$XTZ                DATA
 0002:00000268 00000000H .gehcont$y              DATA
 0002:00000268 00000000H .gfids$y                DATA
 0002:00000270 00002e90H .rdata                  DATA
 0002:00003100 00000000H .rdata$CastGuardVftablesA DATA
 0002:00003100 00000000H .rdata$CastGuardVftablesC DATA
 0002:00003100 00000028H .rdata$T                DATA
 0002:00003128 00000114H .rdata$voltmd           DATA
 0002:0000323c 0000031cH .rdata$zzzdbg           DATA
 0002:00003558 00000008H .rtc$IAA                DATA
 0002:00003560 00000008H .rtc$IZZ                DATA
 0002:00003568 00000008H .rtc$TAA                DATA
 0002:00003570 00000008H .rtc$TZZ                DATA
 0002:00003578 00000004H .tls                    DATA
 0002:0000357c 00000004H .tls$                   DATA
 0002:00003580 00000008H .tls$ZZZ                DATA
 0002:00003588 000003e8H .xdata                  DATA
 0002:00003970 00000368H .edata                  DATA
 0002:00003cd8 0000008cH .idata$2                DATA
 0002:00003d64 00000014H .idata$3                DATA
 0002:00003d78 000001d8H .idata$4                DATA
 0002:00003f50 0000049aH .idata$6                DATA
 0003:00000000 00000080H .data                   DATA
 0003:00000080 0001b258H .bss                    DATA
 0004:00000000 00000438H .pdata                  DATA

  Address         Publics by Value              Rva+Base               Lib:Object

 0000:00000000       __AbsoluteZero             0000000000000000     <absolute>
 0000:00000000       ___safe_se_handler_count   0000000000000000     <absolute>
 0000:00000000       ___safe_se_handler_table   0000000000000000     <absolute>
 0000:00000000       __arm64x_extra_rfe_table   0000000000000000     <absolute>
 0000:00000000       __arm64x_extra_rfe_table_size 0000000000000000     <absolute>
 0000:00000000       __arm64x_native_entrypoint 0000000000000000     <absolute>
 0000:00000000       __arm64x_redirection_metadata 0000000000000000     <absolute>
 0000:00000000       __arm64x_redirection_metadata_count 0000000000000000     <absolute>
 0000:00000000       __dynamic_value_reloc_table 0000000000000000     <absolute>
 0000:00000000       __enclave_config           0000000000000000     <absolute>
 0000:00000000       __guard_check_icall_a64n_fptr 0000000000000000     <absolute>
 0000:00000000       __guard_eh_cont_count      0000000000000000     <absolute>
 0000:00000000       __guard_eh_cont_table      0000000000000000     <absolute>
 0000:00000000       __guard_fids_count         0000000000000000     <absolute>
 0000:00000000       __guard_fids_table         0000000000000000     <absolute>
 0000:00000000       __guard_iat_count          0000000000000000     <absolute>
 0000:00000000       __guard_iat_table          0000000000000000     <absolute>
 0000:00000000       __guard_longjmp_count      0000000000000000     <absolute>
 0000:00000000       __guard_longjmp_table      0000000000000000     <absolute>
 0000:00000000       __hybrid_auxiliary_iat     0000000000000000     <absolute>
 0000:00000000       __hybrid_auxiliary_iat_copy 0000000000000000     <absolute>
 0000:00000000       __hybrid_code_map          0000000000000000     <absolute>
 0000:00000000       __hybrid_code_map_count    0000000000000000     <absolute>
 0000:00000000       __x64_code_ranges_to_entry_points 0000000000000000     <absolute>
 0000:00000000       __x64_code_ranges_to_entry_points_count 0000000000000000     <absolute>
 0000:00000100       __guard_flags              0000000000000100     <absolute>
 0000:00000000       __ImageBase                0000000180000000     <linker-defined>
 0001:00000000       ?NewObject@JNIEnv_@@QEAAPEAV_jobject@@PEAV_jclass@@PEAU_jmethodID@@ZZ 0000000180001000 f i libclassfloadhk007.obj
 0001:00000024       ?SetEventNotificationMode@_jvmtiEnv@@QEAA?AW4jvmtiError@@W4jvmtiEventMode@@W4jvmtiEvent@@PEAV_jobject@@ZZ 0000000180001024 f i libclassfloadhk007.obj
 0001:0000002c       ?TranslateError@@YAPEBDW4jvmtiError@@@Z 000000018000102c f   libclassfloadhk007.obj
 0001:000002e4       ?nsk_jni_check_exception@@YAHPEAUJNIEnv_@@QEBDH@Z 00000001800012e4 f   libclassfloadhk007.obj
 0001:00000428       ?nsk_jni_lverify@@YAHHPEAUJNIEnv_@@HQEBDH1ZZ 0000000180001428 f   libclassfloadhk007.obj
 0001:000004c8       Agent_Initialize           00000001800014c8 f   libclassfloadhk007.obj
 0001:00000788       Agent_OnAttach             0000000180001788 f   libclassfloadhk007.obj
 0001:00000788       Agent_OnLoad               0000000180001788 f   libclassfloadhk007.obj
 0001:00000790       Java_nsk_jvmti_unit_FollowReferences_FollowRefObjects_addRefToVerify 0000000180001790 f   libclassfloadhk007.obj
 0001:0000094c       Java_nsk_jvmti_unit_FollowReferences_FollowRefObjects_getTag 000000018000194c f   libclassfloadhk007.obj
 0001:00000a08       Java_nsk_jvmti_unit_FollowReferences_FollowRefObjects_resetRefsToVerify 0000000180001a08 f   libclassfloadhk007.obj
 0001:00000a10       Java_nsk_jvmti_unit_FollowReferences_FollowRefObjects_resetTags 0000000180001a10 f   libclassfloadhk007.obj
 0001:00000a54       Java_nsk_jvmti_unit_FollowReferences_FollowRefObjects_setTag 0000000180001a54 f   libclassfloadhk007.obj
 0001:00000ca0       Java_nsk_share_jvmti_ArgumentHandler_getAgentOptionsString 0000000180001ca0 f   libclassfloadhk007.obj
 0001:00000d4c       Java_nsk_share_jvmti_DebugeeClass_checkStatus 0000000180001d4c f   libclassfloadhk007.obj
 0001:00000dd4       Java_nsk_share_jvmti_DebugeeClass_resetAgentData 0000000180001dd4 f   libclassfloadhk007.obj
 0001:00000e34       Java_nsk_share_jvmti_RedefineAgent_agentStatus 0000000180001e34 f   libclassfloadhk007.obj
 0001:00000e40       Java_nsk_share_jvmti_RedefineAgent_isRedefined 0000000180001e40 f   libclassfloadhk007.obj
 0001:00000e4c       Java_nsk_share_jvmti_RedefineAgent_redefineAttempted 0000000180001e4c f   libclassfloadhk007.obj
 0001:00000e58       MA_checkStatus             0000000180001e58 f   libclassfloadhk007.obj
 0001:00000efc       __local_stdio_printf_options 0000000180001efc f i libclassfloadhk007.obj
 0001:00001d0c       exitOnError                0000000180002d0c f   libclassfloadhk007.obj
 0001:00001dc0       fprintf                    0000000180002dc0 f i libclassfloadhk007.obj
 0001:0000245c       nsk_complain               000000018000345c f   libclassfloadhk007.obj
 0001:00002488       nsk_jvmti_createJVMTIEnv   0000000180003488 f   libclassfloadhk007.obj
 0001:000025b8       nsk_jvmti_enableEvents     00000001800035b8 f   libclassfloadhk007.obj
 0001:00002694       nsk_jvmti_lverify          0000000180003694 f   libclassfloadhk007.obj
 0001:00002784       nsk_jvmti_parseOptions     0000000180003784 f   libclassfloadhk007.obj
 0001:000029d4       nsk_jvmti_resetAgentData   00000001800039d4 f   libclassfloadhk007.obj
 0001:00002a48       nsk_jvmti_resumeSync       0000000180003a48 f   libclassfloadhk007.obj
 0001:00002aec       nsk_jvmti_waitForSync      0000000180003aec f   libclassfloadhk007.obj
 0001:00002bf0       nsk_lcomplain              0000000180003bf0 f   libclassfloadhk007.obj
 0001:00002c10       nsk_ldisplay               0000000180003c10 f   libclassfloadhk007.obj
 0001:00002c30       nsk_ltrace                 0000000180003c30 f   libclassfloadhk007.obj
 0001:00002c50       nsk_lvcomplain             0000000180003c50 f   libclassfloadhk007.obj
 0001:00002e08       nsk_lvdisplay              0000000180003e08 f   libclassfloadhk007.obj
 0001:00002e54       nsk_lverify                0000000180003e54 f   libclassfloadhk007.obj
 0001:00002eb0       nsk_lvtrace                0000000180003eb0 f   libclassfloadhk007.obj
 0001:00002f10       nsk_printHexBytes          0000000180003f10 f   libclassfloadhk007.obj
 0001:0000307c       nsk_printf                 000000018000407c f   libclassfloadhk007.obj
 0001:000030a4       nsk_vprintf                00000001800040a4 f   libclassfloadhk007.obj
 0001:00003158       printf                     0000000180004158 f i libclassfloadhk007.obj
 0001:000032a8       snprintf                   00000001800042a8 f i libclassfloadhk007.obj
 0001:000037ac       __raise_securityfailure    00000001800047ac f   MSVCRT:gs_report.obj
 0001:000037e0       __report_gsfailure         00000001800047e0 f   MSVCRT:gs_report.obj
 0001:000038b4       __report_rangecheckfailure 00000001800048b4 f   MSVCRT:gs_report.obj
 0001:000038c8       __report_securityfailure   00000001800048c8 f   MSVCRT:gs_report.obj
 0001:00003b40       __GSHandlerCheck           0000000180004b40 f   MSVCRT:gshandler.obj
 0001:00003b60       __GSHandlerCheckCommon     0000000180004b60 f   MSVCRT:gshandler.obj
 0001:00003bd0       __security_check_cookie    0000000180004bd0 f   MSVCRT:amdsecgs.obj
 0001:00003f10       _DllMainCRTStartup         0000000180004f10 f   MSVCRT:dll_dllmain.obj
 0001:00003f50       __scrt_acquire_startup_lock 0000000180004f50 f   MSVCRT:utility.obj
 0001:00003f8c       __scrt_dllmain_after_initialize_c 0000000180004f8c f   MSVCRT:utility.obj
 0001:00003fc0       __scrt_dllmain_before_initialize_c 0000000180004fc0 f   MSVCRT:utility.obj
 0001:00003fd8       __scrt_dllmain_crt_thread_attach 0000000180004fd8 f   MSVCRT:utility.obj
 0001:00004000       __scrt_dllmain_crt_thread_detach 0000000180005000 f   MSVCRT:utility.obj
 0001:00004018       __scrt_dllmain_exception_filter 0000000180005018 f   MSVCRT:utility.obj
 0001:00004078       __scrt_dllmain_uninitialize_c 0000000180005078 f   MSVCRT:utility.obj
 0001:000040a8       __scrt_dllmain_uninitialize_critical 00000001800050a8 f   MSVCRT:utility.obj
 0001:000040bc       __scrt_initialize_crt      00000001800050bc f   MSVCRT:utility.obj
 0001:00004108       __scrt_initialize_onexit_tables 0000000180005108 f   MSVCRT:utility.obj
 0001:00004194       __scrt_is_nonwritable_in_current_image 0000000180005194 f   MSVCRT:utility.obj
 0001:0000422c       __scrt_release_startup_lock 000000018000522c f   MSVCRT:utility.obj
 0001:00004250       __scrt_uninitialize_crt    0000000180005250 f   MSVCRT:utility.obj
 0001:0000427c       _onexit                    000000018000527c f   MSVCRT:utility.obj
 0001:000042b8       atexit                     00000001800052b8 f   MSVCRT:utility.obj
 0001:000042d0       __crt_debugger_hook        00000001800052d0 f   MSVCRT:utility_desktop.obj
 0001:000042d8       __scrt_fastfail            00000001800052d8 f   MSVCRT:utility_desktop.obj
 0001:00004424       _guard_check_icall_nop     0000000180005424 f i MSVCRT:guard_support.obj
 0001:00004428       __security_init_cookie     0000000180005428 f   MSVCRT:gs_support.obj
 0001:000044d4       DllMain                    00000001800054d4 f   MSVCRT:dll_dllmain_stub.obj
 0001:000044f8       ?__scrt_initialize_type_info@@YAXXZ 00000001800054f8 f   MSVCRT:tncleanup.obj
 0001:00004508       ?__scrt_uninitialize_type_info@@YAXXZ 0000000180005508 f   MSVCRT:tncleanup.obj
 0001:00004514       __local_stdio_scanf_options 0000000180005514 f i MSVCRT:default_local_stdio_options.obj
 0001:0000451c       __scrt_initialize_default_local_stdio_options 000000018000551c f   MSVCRT:default_local_stdio_options.obj
 0001:00004538       __scrt_get_dyn_tls_init_callback 0000000180005538 f   MSVCRT:dyn_tls_init.obj
 0001:00004540       _RTC_Initialize            0000000180005540 f   MSVCRT:initsect.obj
 0001:0000457c       _RTC_Terminate             000000018000557c f   MSVCRT:initsect.obj
 0001:000045b8       __isa_available_init       00000001800055b8 f   MSVCRT:cpu_disp.obj
 0001:00004764       _get_startup_argv_mode     0000000180005764 f   MSVCRT:argv_mode.obj
 0001:0000476c       __scrt_is_ucrt_dll_in_use  000000018000576c f   MSVCRT:ucrt_detection.obj
 0001:00004780       memcpy                     0000000180005780 f   vcruntime:VCRUNTIME140.dll
 0001:00004786       memset                     0000000180005786 f   vcruntime:VCRUNTIME140.dll
 0001:0000478c       strchr                     000000018000578c f   vcruntime:VCRUNTIME140.dll
 0001:00004792       __C_specific_handler       0000000180005792 f   vcruntime:VCRUNTIME140.dll
 0001:00004798       __std_type_info_destroy_list 0000000180005798 f   vcruntime:VCRUNTIME140.dll
 0001:0000479e       strcat                     000000018000579e f   ucrt:api-ms-win-crt-string-l1-1-0.dll
 0001:000047a4       strcmp                     00000001800057a4 f   ucrt:api-ms-win-crt-string-l1-1-0.dll
 0001:000047aa       strlen                     00000001800057aa f   ucrt:api-ms-win-crt-string-l1-1-0.dll
 0001:000047b0       _initterm                  00000001800057b0 f   ucrt:api-ms-win-crt-runtime-l1-1-0.dll
 0001:000047b6       _initterm_e                00000001800057b6 f   ucrt:api-ms-win-crt-runtime-l1-1-0.dll
 0001:000047bc       _seh_filter_dll            00000001800057bc f   ucrt:api-ms-win-crt-runtime-l1-1-0.dll
 0001:000047c2       _configure_narrow_argv     00000001800057c2 f   ucrt:api-ms-win-crt-runtime-l1-1-0.dll
 0001:000047c8       _initialize_narrow_environment 00000001800057c8 f   ucrt:api-ms-win-crt-runtime-l1-1-0.dll
 0001:000047ce       _initialize_onexit_table   00000001800057ce f   ucrt:api-ms-win-crt-runtime-l1-1-0.dll
 0001:000047d4       _register_onexit_function  00000001800057d4 f   ucrt:api-ms-win-crt-runtime-l1-1-0.dll
 0001:000047da       _execute_onexit_table      00000001800057da f   ucrt:api-ms-win-crt-runtime-l1-1-0.dll
 0001:000047e0       _crt_atexit                00000001800057e0 f   ucrt:api-ms-win-crt-runtime-l1-1-0.dll
 0001:000047e6       _cexit                     00000001800057e6 f   ucrt:api-ms-win-crt-runtime-l1-1-0.dll
 0001:000047ec       __acrt_initialize          00000001800057ec f   MSVCRT:ucrt_stubs.obj
 0001:000047ec       __acrt_thread_attach       00000001800057ec f   MSVCRT:ucrt_stubs.obj
 0001:000047ec       __acrt_thread_detach       00000001800057ec f   MSVCRT:ucrt_stubs.obj
 0001:000047ec       __acrt_uninitialize        00000001800057ec f   MSVCRT:ucrt_stubs.obj
 0001:000047ec       __acrt_uninitialize_critical 00000001800057ec f   MSVCRT:ucrt_stubs.obj
 0001:000047ec       __scrt_stub_for_acrt_initialize 00000001800057ec f   MSVCRT:ucrt_stubs.obj
 0001:000047ec       __scrt_stub_for_acrt_thread_attach 00000001800057ec f   MSVCRT:ucrt_stubs.obj
 0001:000047ec       __scrt_stub_for_acrt_thread_detach 00000001800057ec f   MSVCRT:ucrt_stubs.obj
 0001:000047ec       __scrt_stub_for_acrt_uninitialize 00000001800057ec f   MSVCRT:ucrt_stubs.obj
 0001:000047ec       __scrt_stub_for_acrt_uninitialize_critical 00000001800057ec f   MSVCRT:ucrt_stubs.obj
 0001:000047ec       __vcrt_initialize          00000001800057ec f   MSVCRT:ucrt_stubs.obj
 0001:000047ec       __vcrt_thread_attach       00000001800057ec f   MSVCRT:ucrt_stubs.obj
 0001:000047ec       __vcrt_thread_detach       00000001800057ec f   MSVCRT:ucrt_stubs.obj
 0001:000047ec       __vcrt_uninitialize        00000001800057ec f   MSVCRT:ucrt_stubs.obj
 0001:000047ec       __vcrt_uninitialize_critical 00000001800057ec f   MSVCRT:ucrt_stubs.obj
 0001:000047f0       __scrt_stub_for_is_c_termination_complete 00000001800057f0 f   MSVCRT:ucrt_stubs.obj
 0001:000047f0       _is_c_termination_complete 00000001800057f0 f   MSVCRT:ucrt_stubs.obj
 0001:00004810       _guard_dispatch_icall_nop  0000000180005810 f   MSVCRT:guard_dispatch.obj
 0001:00004830       _guard_xfg_dispatch_icall_nop 0000000180005830 f   MSVCRT:guard_xfg_dispatch.obj
 0002:00000000       __imp_RtlCaptureContext    0000000180006000     kernel32:KERNEL32.dll
 0002:00000008       __imp_RtlLookupFunctionEntry 0000000180006008     kernel32:KERNEL32.dll
 0002:00000010       __imp_RtlVirtualUnwind     0000000180006010     kernel32:KERNEL32.dll
 0002:00000018       __imp_UnhandledExceptionFilter 0000000180006018     kernel32:KERNEL32.dll
 0002:00000020       __imp_SetUnhandledExceptionFilter 0000000180006020     kernel32:KERNEL32.dll
 0002:00000028       __imp_GetCurrentProcess    0000000180006028     kernel32:KERNEL32.dll
 0002:00000030       __imp_TerminateProcess     0000000180006030     kernel32:KERNEL32.dll
 0002:00000038       __imp_IsProcessorFeaturePresent 0000000180006038     kernel32:KERNEL32.dll
 0002:00000040       __imp_CloseHandle          0000000180006040     kernel32:KERNEL32.dll
 0002:00000048       __imp_InitializeCriticalSectionAndSpinCount 0000000180006048     kernel32:KERNEL32.dll
 0002:00000050       __imp_DeleteCriticalSection 0000000180006050     kernel32:KERNEL32.dll
 0002:00000058       __imp_CreateEventW         0000000180006058     kernel32:KERNEL32.dll
 0002:00000060       __imp_GetModuleHandleW     0000000180006060     kernel32:KERNEL32.dll
 0002:00000068       __imp_GetProcAddress       0000000180006068     kernel32:KERNEL32.dll
 0002:00000070       __imp_IsDebuggerPresent    0000000180006070     kernel32:KERNEL32.dll
 0002:00000078       __imp_QueryPerformanceCounter 0000000180006078     kernel32:KERNEL32.dll
 0002:00000080       __imp_GetCurrentProcessId  0000000180006080     kernel32:KERNEL32.dll
 0002:00000088       __imp_GetCurrentThreadId   0000000180006088     kernel32:KERNEL32.dll
 0002:00000090       __imp_GetSystemTimeAsFileTime 0000000180006090     kernel32:KERNEL32.dll
 0002:00000098       __imp_DisableThreadLibraryCalls 0000000180006098     kernel32:KERNEL32.dll
 0002:000000a0       __imp_InitializeSListHead  00000001800060a0     kernel32:KERNEL32.dll
 0002:000000a8       \177KERNEL32_NULL_THUNK_DATA 00000001800060a8     kernel32:KERNEL32.dll
 0002:000000b0       __imp_memcpy               00000001800060b0     vcruntime:VCRUNTIME140.dll
 0002:000000b8       __imp_memset               00000001800060b8     vcruntime:VCRUNTIME140.dll
 0002:000000c0       __imp_strchr               00000001800060c0     vcruntime:VCRUNTIME140.dll
 0002:000000c8       __imp___C_specific_handler 00000001800060c8     vcruntime:VCRUNTIME140.dll
 0002:000000d0       __imp___std_type_info_destroy_list 00000001800060d0     vcruntime:VCRUNTIME140.dll
 0002:000000d8       \177VCRUNTIME140_NULL_THUNK_DATA 00000001800060d8     vcruntime:VCRUNTIME140.dll
 0002:000000e0       __imp_strtol               00000001800060e0     ucrt:api-ms-win-crt-convert-l1-1-0.dll
 0002:000000e8       \177api-ms-win-crt-convert-l1-1-0_NULL_THUNK_DATA 00000001800060e8     ucrt:api-ms-win-crt-convert-l1-1-0.dll
 0002:000000f0       __imp_malloc               00000001800060f0     ucrt:api-ms-win-crt-heap-l1-1-0.dll
 0002:000000f8       __imp_free                 00000001800060f8     ucrt:api-ms-win-crt-heap-l1-1-0.dll
 0002:00000100       \177api-ms-win-crt-heap-l1-1-0_NULL_THUNK_DATA 0000000180006100     ucrt:api-ms-win-crt-heap-l1-1-0.dll
 0002:00000108       __imp__errno               0000000180006108     ucrt:api-ms-win-crt-runtime-l1-1-0.dll
 0002:00000110       __imp_exit                 0000000180006110     ucrt:api-ms-win-crt-runtime-l1-1-0.dll
 0002:00000118       __imp__cexit               0000000180006118     ucrt:api-ms-win-crt-runtime-l1-1-0.dll
 0002:00000120       __imp__crt_atexit          0000000180006120     ucrt:api-ms-win-crt-runtime-l1-1-0.dll
 0002:00000128       __imp__execute_onexit_table 0000000180006128     ucrt:api-ms-win-crt-runtime-l1-1-0.dll
 0002:00000130       __imp__register_onexit_function 0000000180006130     ucrt:api-ms-win-crt-runtime-l1-1-0.dll
 0002:00000138       __imp__initialize_onexit_table 0000000180006138     ucrt:api-ms-win-crt-runtime-l1-1-0.dll
 0002:00000140       __imp__initialize_narrow_environment 0000000180006140     ucrt:api-ms-win-crt-runtime-l1-1-0.dll
 0002:00000148       __imp__configure_narrow_argv 0000000180006148     ucrt:api-ms-win-crt-runtime-l1-1-0.dll
 0002:00000150       __imp__seh_filter_dll      0000000180006150     ucrt:api-ms-win-crt-runtime-l1-1-0.dll
 0002:00000158       __imp__initterm_e          0000000180006158     ucrt:api-ms-win-crt-runtime-l1-1-0.dll
 0002:00000160       __imp__initterm            0000000180006160     ucrt:api-ms-win-crt-runtime-l1-1-0.dll
 0002:00000168       \177api-ms-win-crt-runtime-l1-1-0_NULL_THUNK_DATA 0000000180006168     ucrt:api-ms-win-crt-runtime-l1-1-0.dll
 0002:00000170       __imp___acrt_iob_func      0000000180006170     ucrt:api-ms-win-crt-stdio-l1-1-0.dll
 0002:00000178       __imp_fflush               0000000180006178     ucrt:api-ms-win-crt-stdio-l1-1-0.dll
 0002:00000180       __imp___stdio_common_vsprintf 0000000180006180     ucrt:api-ms-win-crt-stdio-l1-1-0.dll
 0002:00000188       __imp___stdio_common_vfprintf 0000000180006188     ucrt:api-ms-win-crt-stdio-l1-1-0.dll
 0002:00000190       \177api-ms-win-crt-stdio-l1-1-0_NULL_THUNK_DATA 0000000180006190     ucrt:api-ms-win-crt-stdio-l1-1-0.dll
 0002:00000198       __imp_strcat               0000000180006198     ucrt:api-ms-win-crt-string-l1-1-0.dll
 0002:000001a0       __imp_strcmp               00000001800061a0     ucrt:api-ms-win-crt-string-l1-1-0.dll
 0002:000001a8       __imp__strdup              00000001800061a8     ucrt:api-ms-win-crt-string-l1-1-0.dll
 0002:000001a8       __imp_strdup               00000001800061a8     ucrt:api-ms-win-crt-string-l1-1-0.dll
 0002:000001b0       __imp_strlen               00000001800061b0     ucrt:api-ms-win-crt-string-l1-1-0.dll
 0002:000001b8       __imp_strpbrk              00000001800061b8     ucrt:api-ms-win-crt-string-l1-1-0.dll
 0002:000001c0       __imp_strncpy              00000001800061c0     ucrt:api-ms-win-crt-string-l1-1-0.dll
 0002:000001c8       __imp_isprint              00000001800061c8     ucrt:api-ms-win-crt-string-l1-1-0.dll
 0002:000001d0       \177api-ms-win-crt-string-l1-1-0_NULL_THUNK_DATA 00000001800061d0     ucrt:api-ms-win-crt-string-l1-1-0.dll
 0002:000001d8       __guard_check_icall_fptr   00000001800061d8     MSVCRT:guard_support.obj
 0002:000001e0       __guard_xfg_check_icall_fptr 00000001800061e0     MSVCRT:guard_support.obj
 0002:000001e8       __guard_dispatch_icall_fptr 00000001800061e8     MSVCRT:guard_support.obj
 0002:000001f0       __guard_xfg_dispatch_icall_fptr 00000001800061f0     MSVCRT:guard_support.obj
 0002:000001f8       __guard_xfg_table_dispatch_icall_fptr 00000001800061f8     MSVCRT:guard_support.obj
 0002:00000200       __castguard_check_failure_os_handled_fptr 0000000180006200     MSVCRT:guard_support.obj
 0002:00000208       __guard_memcpy_fptr        0000000180006208     vcruntime:softmemtag.obj
 0002:00000210       __xc_a                     0000000180006210     MSVCRT:initializers.obj
 0002:00000218       __xc_z                     0000000180006218     MSVCRT:initializers.obj
 0002:00000220       __xi_a                     0000000180006220     MSVCRT:initializers.obj
 0002:00000230       __xi_z                     0000000180006230     MSVCRT:initializers.obj
 0002:00000238       __xl_a                     0000000180006238     MSVCRT:tlssup.obj
 0002:00000240       __xl_z                     0000000180006240     MSVCRT:tlssup.obj
 0002:00000248       __xp_a                     0000000180006248     MSVCRT:initializers.obj
 0002:00000250       __xp_z                     0000000180006250     MSVCRT:initializers.obj
 0002:00000258       __xt_a                     0000000180006258     MSVCRT:initializers.obj
 0002:00000260       __xt_z                     0000000180006260     MSVCRT:initializers.obj
 0002:00000270       g_refKindStr               0000000180006270     libclassfloadhk007.obj
 0002:00000420       ??_C@_09BPLDFGCI@unknown_0@ 0000000180006420     libclassfloadhk007.obj
 0002:00000430       ??_C@_0BL@FPNMECJD@JVMTI_HEAP_REFERENCE_CLASS@ 0000000180006430     libclassfloadhk007.obj
 0002:00000450       ??_C@_0BL@FKGKKLNM@JVMTI_HEAP_REFERENCE_FIELD@ 0000000180006450     libclassfloadhk007.obj
 0002:00000470       ??_C@_0CD@CAEHCFJF@JVMTI_HEAP_REFERENCE_ARRAY_ELEM@ 0000000180006470     libclassfloadhk007.obj
 0002:00000498       ??_C@_0CC@DNEBMCNK@JVMTI_HEAP_REFERENCE_CLASS_LOAD@ 0000000180006498     libclassfloadhk007.obj
 0002:000004c0       ??_C@_0BN@CJMIPEBB@JVMTI_HEAP_REFERENCE_SIGNERS@ 00000001800064c0     libclassfloadhk007.obj
 0002:000004e0       ??_C@_0CH@HBOIDPEB@JVMTI_HEAP_REFERENCE_PROTECTION@ 00000001800064e0     libclassfloadhk007.obj
 0002:00000508       ??_C@_0BP@MDKGDGKL@JVMTI_HEAP_REFERENCE_INTERFACE@ 0000000180006508     libclassfloadhk007.obj
 0002:00000528       ??_C@_0CC@JJMIHNJH@JVMTI_HEAP_REFERENCE_STATIC_FIE@ 0000000180006528     libclassfloadhk007.obj
 0002:00000550       ??_C@_0CD@IDHEEGID@JVMTI_HEAP_REFERENCE_CONSTANT_P@ 0000000180006550     libclassfloadhk007.obj
 0002:00000578       ??_C@_0CA@EFFCHNG@JVMTI_HEAP_REFERENCE_SUPERCLASS@ 0000000180006578     libclassfloadhk007.obj
 0002:00000598       ??_C@_0L@PCDFHGCJ@unknown_11@ 0000000180006598     libclassfloadhk007.obj
 0002:000005a8       ??_C@_0L@NJBICFOK@unknown_12@ 00000001800065a8     libclassfloadhk007.obj
 0002:000005b8       ??_C@_0L@MAADBEKL@unknown_13@ 00000001800065b8     libclassfloadhk007.obj
 0002:000005c8       ??_C@_0L@IPECICGM@unknown_14@ 00000001800065c8     libclassfloadhk007.obj
 0002:000005d8       ??_C@_0L@JGFJLDCN@unknown_15@ 00000001800065d8     libclassfloadhk007.obj
 0002:000005e8       ??_C@_0L@LNHEOAOO@unknown_16@ 00000001800065e8     libclassfloadhk007.obj
 0002:000005f8       ??_C@_0L@KEGPNBKP@unknown_17@ 00000001800065f8     libclassfloadhk007.obj
 0002:00000608       ??_C@_0L@CDPHMNGA@unknown_18@ 0000000180006608     libclassfloadhk007.obj
 0002:00000618       ??_C@_0L@DKOMPMCB@unknown_19@ 0000000180006618     libclassfloadhk007.obj
 0002:00000628       ??_C@_0L@OJGIPJDB@unknown_20@ 0000000180006628     libclassfloadhk007.obj
 0002:00000638       ??_C@_0CA@KAOFNDEM@JVMTI_HEAP_REFERENCE_JNI_GLOBAL@ 0000000180006638     libclassfloadhk007.obj
 0002:00000658       ??_C@_0CC@HPFAJBK@JVMTI_HEAP_REFERENCE_SYSTEM_CLA@ 0000000180006658     libclassfloadhk007.obj
 0002:00000680       ??_C@_0BN@FDEGFOHC@JVMTI_HEAP_REFERENCE_MONITOR@ 0000000180006680     libclassfloadhk007.obj
 0002:000006a0       ??_C@_0CB@HKIBCMAJ@JVMTI_HEAP_REFERENCE_STACK_LOCA@ 00000001800066a0     libclassfloadhk007.obj
 0002:000006c8       ??_C@_0BP@EAACMMOE@JVMTI_HEAP_REFERENCE_JNI_LOCAL@ 00000001800066c8     libclassfloadhk007.obj
 0002:000006e8       ??_C@_0BM@IJDEOGOE@JVMTI_HEAP_REFERENCE_THREAD@ 00000001800066e8     libclassfloadhk007.obj
 0002:00000708       ??_C@_0BL@EDGPPKC@JVMTI_HEAP_REFERENCE_OTHER@ 0000000180006708     libclassfloadhk007.obj
 0002:00000724       ??_C@_04BCJPDBDA@Code@     0000000180006724     libclassfloadhk007.obj
 0002:00000730       ??_C@_0BA@OCLMCFKC@LineNumberTable@ 0000000180006730     libclassfloadhk007.obj
 0002:00000740       ??_C@_0BD@CPAEPILC@LocalVariableTable@ 0000000180006740     libclassfloadhk007.obj
 0002:00000758       ??_C@_0BH@NMBDNHBD@LocalVariableTypeTable@ 0000000180006758     libclassfloadhk007.obj
 0002:00000770       ??_C@_0O@HIHEEDNJ@StackMapTable@ 0000000180006770     libclassfloadhk007.obj
 0002:00000780       ??_C@_0L@HCDIAMJG@?9?5?$CFs?0?5?$CFd?3?5@ 0000000180006780     libclassfloadhk007.obj
 0002:00000790       ??_C@_0JI@HLPECLFI@?$CD?5?4?4?4?6?$CD?5ERROR?3?5too?5many?5complai@ 0000000180006790     libclassfloadhk007.obj
 0002:00000830       ??_C@_0ED@JNEKCCOB@The?5following?5fake?5exception?5st@ 0000000180006830     libclassfloadhk007.obj
 0002:00000878       ??_C@_0CN@FCNMDFBH@nsk?4share?4Fake_Exception_for_RU@ 0000000180006878     libclassfloadhk007.obj
 0002:000008a8       ??_C@_08PGFFNAEI@?$CI?$CFs?3?$CFd?$CJ?5@ 00000001800068a8     libclassfloadhk007.obj
 0002:000008b8       ??_C@_0DP@IENMAEGI@s?2test?2hotspot?2jtreg?2vmTestbase@ 00000001800068b8     libclassfloadhk007.obj
 0002:000008f8       ??_C@_0BL@NDJLFFJB@?7at?5nsk_lvcomplain?$CI?$CFs?3?$CFd?$CJ?6@ 00000001800068f8     libclassfloadhk007.obj
 0002:00000918       ??_C@_0BC@JOOKAFKF@?$CD?5ERROR?3?5?$CFs?0?5?$CFd?3?5@ 0000000180006918     libclassfloadhk007.obj
 0002:00000930       ??_C@_09KJEAHMEH@?$CD?5ERROR?3?5@ 0000000180006930     libclassfloadhk007.obj
 0002:0000093c       ??_C@_02GPIOPFAK@?$DO?$DO@ 000000018000693c     libclassfloadhk007.obj
 0002:00000940       ??_C@_02FODMEDOG@?$DM?$DM@ 0000000180006940     libclassfloadhk007.obj
 0002:00000944       ??_C@_02DJGKEECL@?4?4@     0000000180006944     libclassfloadhk007.obj
 0002:00000948       ??_C@_0O@CJPGJOAF@?9?5?$CFs?0?5?$CFd?3?5?$CFs?5@ 0000000180006948     libclassfloadhk007.obj
 0002:00000958       ??_C@_0CB@IAKPDOIC@?$CD?5?5?5verified?5assertion?5is?5FALSE@ 0000000180006958     libclassfloadhk007.obj
 0002:00000980       ??_C@_0CO@LGONDEPD@stdout?3?5fflush?5failed?5?9?5err?$DN?$CFd?5@ 0000000180006980     libclassfloadhk007.obj
 0002:000009b0       ??_C@_0CO@KBGKJPBD@stderr?3?5fflush?5failed?5?9?5err?$DN?$CFd?5@ 00000001800069b0     libclassfloadhk007.obj
 0002:000009e0       ??_C@_05OFBGOFBN@?5?$CF02X@ 00000001800069e0     libclassfloadhk007.obj
 0002:000009e8       ??_C@_03NDEAONJP@?5?5?5@   00000001800069e8     libclassfloadhk007.obj
 0002:000009f0       ??_C@_0BF@BLCOCCJM@?$CFs0x?$CF08X?3?5?5?$CFs?5?5?5?5?$CFs?6@ 00000001800069f0     libclassfloadhk007.obj
 0002:00000a08       ??_C@_06HPGEIPLA@?$DMnull?$DO@ 0000000180006a08     libclassfloadhk007.obj
 0002:00000a10       ??_C@_0BB@JCNMKLLK@JVMTI_ERROR_NONE@ 0000000180006a10     libclassfloadhk007.obj
 0002:00000a28       ??_C@_0BL@LDIMKLPH@JVMTI_ERROR_INVALID_THREAD@ 0000000180006a28     libclassfloadhk007.obj
 0002:00000a48       ??_C@_0CB@PJFPAIKJ@JVMTI_ERROR_INVALID_THREAD_GROU@ 0000000180006a48     libclassfloadhk007.obj
 0002:00000a70       ??_C@_0BN@LLMKHMNF@JVMTI_ERROR_INVALID_PRIORITY@ 0000000180006a70     libclassfloadhk007.obj
 0002:00000a90       ??_C@_0CB@MBOFKAGB@JVMTI_ERROR_THREAD_NOT_SUSPENDE@ 0000000180006a90     libclassfloadhk007.obj
 0002:00000ab8       ??_C@_0BN@FABOLPBI@JVMTI_ERROR_THREAD_SUSPENDED@ 0000000180006ab8     libclassfloadhk007.obj
 0002:00000ad8       ??_C@_0BN@FDGNOBJM@JVMTI_ERROR_THREAD_NOT_ALIVE@ 0000000180006ad8     libclassfloadhk007.obj
 0002:00000af8       ??_C@_0BL@GOBIFKNJ@JVMTI_ERROR_INVALID_OBJECT@ 0000000180006af8     libclassfloadhk007.obj
 0002:00000b18       ??_C@_0BK@FCMAJPPC@JVMTI_ERROR_INVALID_CLASS@ 0000000180006b18     libclassfloadhk007.obj
 0002:00000b38       ??_C@_0BP@IKLLBKEB@JVMTI_ERROR_CLASS_NOT_PREPARED@ 0000000180006b38     libclassfloadhk007.obj
 0002:00000b58       ??_C@_0BN@KLPPLKG@JVMTI_ERROR_INVALID_METHODID@ 0000000180006b58     libclassfloadhk007.obj
 0002:00000b78       ??_C@_0BN@BCEKOKND@JVMTI_ERROR_INVALID_LOCATION@ 0000000180006b78     libclassfloadhk007.obj
 0002:00000b98       ??_C@_0BM@DFDGPME@JVMTI_ERROR_INVALID_FIELDID@ 0000000180006b98     libclassfloadhk007.obj
 0002:00000bb8       ??_C@_0BL@NELIEPEC@JVMTI_ERROR_NO_MORE_FRAMES@ 0000000180006bb8     libclassfloadhk007.obj
 0002:00000bd8       ??_C@_0BJ@BDBECFDM@JVMTI_ERROR_OPAQUE_FRAME@ 0000000180006bd8     libclassfloadhk007.obj
 0002:00000bf8       ??_C@_0BK@MIIFNLOB@JVMTI_ERROR_TYPE_MISMATCH@ 0000000180006bf8     libclassfloadhk007.obj
 0002:00000c18       ??_C@_0BJ@HPCAOILC@JVMTI_ERROR_INVALID_SLOT@ 0000000180006c18     libclassfloadhk007.obj
 0002:00000c38       ??_C@_0BG@CHILOPNI@JVMTI_ERROR_DUPLICATE@ 0000000180006c38     libclassfloadhk007.obj
 0002:00000c50       ??_C@_0BG@DIEMLHKM@JVMTI_ERROR_NOT_FOUND@ 0000000180006c50     libclassfloadhk007.obj
 0002:00000c68       ??_C@_0BM@NHMCKHOB@JVMTI_ERROR_INVALID_MONITOR@ 0000000180006c68     libclassfloadhk007.obj
 0002:00000c88       ??_C@_0BO@PPEDAJGL@JVMTI_ERROR_NOT_MONITOR_OWNER@ 0000000180006c88     libclassfloadhk007.obj
 0002:00000ca8       ??_C@_0BG@FCAIPEID@JVMTI_ERROR_INTERRUPT@ 0000000180006ca8     libclassfloadhk007.obj
 0002:00000cc0       ??_C@_0CB@EGDBNKOI@JVMTI_ERROR_INVALID_CLASS_FORMA@ 0000000180006cc0     libclassfloadhk007.obj
 0002:00000ce8       ??_C@_0CG@DGKOGIAL@JVMTI_ERROR_CIRCULAR_CLASS_DEFI@ 0000000180006ce8     libclassfloadhk007.obj
 0002:00000d10       ??_C@_0BP@ICEALPKC@JVMTI_ERROR_FAILS_VERIFICATION@ 0000000180006d10     libclassfloadhk007.obj
 0002:00000d30       ??_C@_0DC@JDACLMIO@JVMTI_ERROR_UNSUPPORTED_REDEFIN@ 0000000180006d30     libclassfloadhk007.obj
 0002:00000d68       ??_C@_0DE@GKDKNOMJ@JVMTI_ERROR_UNSUPPORTED_REDEFIN@ 0000000180006d68     libclassfloadhk007.obj
 0002:00000da0       ??_C@_0BO@LAFKIOG@JVMTI_ERROR_INVALID_TYPESTATE@ 0000000180006da0     libclassfloadhk007.obj
 0002:00000dc0       ??_C@_0DH@INDGCLLB@JVMTI_ERROR_UNSUPPORTED_REDEFIN@ 0000000180006dc0     libclassfloadhk007.obj
 0002:00000df8       ??_C@_0DE@NHEOMMGI@JVMTI_ERROR_UNSUPPORTED_REDEFIN@ 0000000180006df8     libclassfloadhk007.obj
 0002:00000e30       ??_C@_0CA@EKPNJOEP@JVMTI_ERROR_UNSUPPORTED_VERSION@ 0000000180006e30     libclassfloadhk007.obj
 0002:00000e50       ??_C@_0BN@OFFMAHHL@JVMTI_ERROR_NAMES_DONT_MATCH@ 0000000180006e50     libclassfloadhk007.obj
 0002:00000e70       ??_C@_0DN@HHBBLAKE@JVMTI_ERROR_UNSUPPORTED_REDEFIN@ 0000000180006e70     libclassfloadhk007.obj
 0002:00000eb0       ??_C@_0DO@HMBGBGNA@JVMTI_ERROR_UNSUPPORTED_REDEFIN@ 0000000180006eb0     libclassfloadhk007.obj
 0002:00000ef0       ??_C@_0BP@PBECGKHJ@JVMTI_ERROR_UNMODIFIABLE_CLASS@ 0000000180006ef0     libclassfloadhk007.obj
 0002:00000f10       ??_C@_0BK@CANILEHF@JVMTI_ERROR_NOT_AVAILABLE@ 0000000180006f10     libclassfloadhk007.obj
 0002:00000f30       ??_C@_0CE@INJKMEFK@JVMTI_ERROR_MUST_POSSESS_CAPABI@ 0000000180006f30     libclassfloadhk007.obj
 0002:00000f58       ??_C@_0BJ@LBFPFPDM@JVMTI_ERROR_NULL_POINTER@ 0000000180006f58     libclassfloadhk007.obj
 0002:00000f78       ??_C@_0BP@CHJPNNEM@JVMTI_ERROR_ABSENT_INFORMATION@ 0000000180006f78     libclassfloadhk007.obj
 0002:00000f98       ??_C@_0BP@OMFMNLC@JVMTI_ERROR_INVALID_EVENT_TYPE@ 0000000180006f98     libclassfloadhk007.obj
 0002:00000fb8       ??_C@_0BN@BIBNPHHO@JVMTI_ERROR_ILLEGAL_ARGUMENT@ 0000000180006fb8     libclassfloadhk007.obj
 0002:00000fd8       ??_C@_0BK@KKNDHDCE@JVMTI_ERROR_NATIVE_METHOD@ 0000000180006fd8     libclassfloadhk007.obj
 0002:00000ff8       ??_C@_0BK@PMKCFHAE@JVMTI_ERROR_OUT_OF_MEMORY@ 0000000180006ff8     libclassfloadhk007.obj
 0002:00001018       ??_C@_0BK@NNJBDMNB@JVMTI_ERROR_ACCESS_DENIED@ 0000000180007018     libclassfloadhk007.obj
 0002:00001038       ??_C@_0BI@GHECLMNC@JVMTI_ERROR_WRONG_PHASE@ 0000000180007038     libclassfloadhk007.obj
 0002:00001050       ??_C@_0BF@OLIHJOII@JVMTI_ERROR_INTERNAL@ 0000000180007050     libclassfloadhk007.obj
 0002:00001068       ??_C@_0BO@EOHGKJHI@JVMTI_ERROR_UNATTACHED_THREAD@ 0000000180007068     libclassfloadhk007.obj
 0002:00001088       ??_C@_0CA@LKHFDACL@JVMTI_ERROR_INVALID_ENVIRONMENT@ 0000000180007088     libclassfloadhk007.obj
 0002:000010a8       ??_C@_0BA@MMFHLOKK@?$DMunknown?5error?$DO@ 00000001800070a8     libclassfloadhk007.obj
 0002:000010b8       ??_C@_0CF@CBHOKDB@throwable?5?$DN?5jni?9?$DOExceptionOccur@ 00000001800070b8     libclassfloadhk007.obj
 0002:000010e0       ??_C@_03OFAPEBGM@?$CFs?6@  00000001800070e0     libclassfloadhk007.obj
 0002:000010e8       ??_C@_0DM@LPIGEGNJ@s?2test?2hotspot?2jtreg?2vmTestbase@ 00000001800070e8     libclassfloadhk007.obj
 0002:00001128       ??_C@_0CC@NFCNPEPK@Exception?5in?5JNI?5call?5?$CIcleared?$CJ@ 0000000180007128     libclassfloadhk007.obj
 0002:00001150       ??_C@_0BJ@IBAKFIKF@jni?9?$DOExceptionDescribe?$CI?$CJ@ 0000000180007150     libclassfloadhk007.obj
 0002:00001170       ??_C@_0BG@GGKALKMH@jni?9?$DOExceptionClear?$CI?$CJ@ 0000000180007170     libclassfloadhk007.obj
 0002:00001188       ??_C@_0CF@JMGFGJLJ@?$CD?5?5?5verified?5JNI?5assertion?5is?5F@ 0000000180007188     libclassfloadhk007.obj
 0002:000011b0       ??_C@_07KBAMPNJK@verbose@  00000001800071b0     libclassfloadhk007.obj
 0002:000011b8       ??_C@_0DN@PKJBOLAP@nsk_jvmti_parseOptions?$CI?$CJ?3?5unexp@ 00000001800071b8     libclassfloadhk007.obj
 0002:000011f8       ??_C@_05IMBNNINJ@trace@    00000001800071f8     libclassfloadhk007.obj
 0002:00001200       ??_C@_0DD@BJKGNDMB@nsk_jvmti_parseOptions?$CI?$CJ?3?5no?5va@ 0000000180007200     libclassfloadhk007.obj
 0002:00001234       ??_C@_04CGFJFPFD@none@     0000000180007234     libclassfloadhk007.obj
 0002:0000123c       ??_C@_06BMELKFMA@before@   000000018000723c     libclassfloadhk007.obj
 0002:00001244       ??_C@_05CMKPCFDK@after@    0000000180007244     libclassfloadhk007.obj
 0002:0000124c       ??_C@_03NFKEKGGK@all@      000000018000724c     libclassfloadhk007.obj
 0002:00001250       ??_C@_0DM@NDNJGJKE@nsk_jvmti_parseOptions?$CI?$CJ?3?5uexpe@ 0000000180007250     libclassfloadhk007.obj
 0002:00001290       ??_C@_08NBBJKJO@waittime@  0000000180007290     libclassfloadhk007.obj
 0002:000012a0       ??_C@_0DO@CMHGAOHC@nsk_jvmti_parseOptions?$CI?$CJ?3?5not?5i@ 00000001800072a0     libclassfloadhk007.obj
 0002:000012e0       ??_C@_0DL@LNMPBDLN@nsk_jvmti_parseOptions?$CI?$CJ?3?5negat@ 00000001800072e0     libclassfloadhk007.obj
 0002:00001320       ??_C@_0DA@GMFJNOJH@nsk_jvmti_parseOptions?$CI?$CJ?3?5unkno@ 0000000180007320     libclassfloadhk007.obj
 0002:00001350       ??_C@_0CO@CCIAMEAN@nsk_jvmti_parseOptions?$CI?$CJ?3?5found@ 0000000180007350     libclassfloadhk007.obj
 0002:00001380       ??_C@_0CJ@OEGPCGDL@nsk_jvmti_parseOptions?$CI?$CJ?3?5out?5o@ 0000000180007380     libclassfloadhk007.obj
 0002:000013b0       ??_C@_0DI@NMBHPGGF@nsk_jvmti_parseOptions?$CI?$CJ?3?5too?5m@ 00000001800073b0     libclassfloadhk007.obj
 0002:000013e8       ??_C@_03POGCGECB@?5?0?$HO@ 00000001800073e8     libclassfloadhk007.obj
 0002:000013f0       ??_C@_0CB@MLNJNCLJ@?5?5jvmti?5error?3?5code?$DN?$CFd?0?5name?$DN?$CFs@ 00000001800073f0     libclassfloadhk007.obj
 0002:00001418       ??_C@_0CD@OHBGDKMK@?$CD?5?5?5jvmti?5error?3?5code?$DN?$CFd?0?5name?$DN@ 0000000180007418     libclassfloadhk007.obj
 0002:00001440       ??_C@_0CG@JNNCGPHB@?$CD?5?5?5error?5expected?3?5code?$DN?$CFd?0?5na@ 0000000180007440     libclassfloadhk007.obj
 0002:00001470       ??_C@_0EB@IMGKPCGE@?$CIstr_obj?5?$DN?5jni?9?$DONewStringUTF?$CIco@ 0000000180007470     libclassfloadhk007.obj
 0002:000014c0       ??_C@_0EA@HFOGGBCC@s?2test?2hotspot?2jtreg?2vmTestbase@ 00000001800074c0     libclassfloadhk007.obj
 0002:00001500       ??_C@_05KKCIMGE@error@     0000000180007500     libclassfloadhk007.obj
 0002:00001508       ??_C@_0BD@HGNAOMCP@agent_data_monitor@ 0000000180007508     libclassfloadhk007.obj
 0002:00001520       ??_C@_0EB@OGCLGKLN@javaVM?9?$DOGetEnv?$CI?$CIvoid?5?$CK?$CK?$CJ?$CGjvmti_@ 0000000180007520     libclassfloadhk007.obj
 0002:00001570       ??_C@_0EA@PNBCDMOA@s?2test?2hotspot?2jtreg?2vmTestbase@ 0000000180007570     libclassfloadhk007.obj
 0002:000015b0       ??_C@_0CI@DDPIFBGM@init_agent_data?$CIjvmti_env?0?5?$CGage@ 00000001800075b0     libclassfloadhk007.obj
 0002:000015d8       ??_C@_0DI@ILAHDLMP@?$CI?$CKagentThreadProc?$CJ?$CIjvmti_env?0?5a@ 00000001800075d8     libclassfloadhk007.obj
 0002:00001610       ??_C@_0BD@KDBALNLB@JVMTI?5agent?5thread@ 0000000180007610     libclassfloadhk007.obj
 0002:00001628       ??_C@_0BB@NOKBFPFO@java?1lang?1Thread@ 0000000180007628     libclassfloadhk007.obj
 0002:0000163c       ??_C@_06FALKBLGB@?$DMinit?$DO@ 000000018000763c     libclassfloadhk007.obj
 0002:00001648       ??_C@_0BG@IKDDPPGD@?$CILjava?1lang?1String?$DL?$CJV@ 0000000180007648     libclassfloadhk007.obj
 0002:00001660       ??_C@_0EB@IFJBFEKC@?$CIthreadClass?5?$DN?5jni_env?9?$DOFindCla@ 0000000180007660     libclassfloadhk007.obj
 0002:000016b0       ??_C@_0GF@FGFIBKKL@?$CIthreadCtor?5?$DN?5jni_env?9?$DOGetMetho@ 00000001800076b0     libclassfloadhk007.obj
 0002:00001718       ??_C@_0DN@NCPDJLOG@?$CIthreadName?5?$DN?5jni_env?9?$DONewStrin@ 0000000180007718     libclassfloadhk007.obj
 0002:00001760       ??_C@_0FE@PFKODBGC@?$CIthreadObject?5?$DN?5jni_env?9?$DONewObj@ 0000000180007760     libclassfloadhk007.obj
 0002:000017c0       ??_C@_0ED@HOBAHHJI@?$CIthreadGlobalRef?5?$DN?5jni_env?9?$DONew@ 00000001800077c0     libclassfloadhk007.obj
 0002:00001810       ??_C@_0FN@HNJJAHFC@jvmti_env?9?$DORunAgentThread?$CIagent@ 0000000180007810     libclassfloadhk007.obj
 0002:00001870       ??_C@_0EA@MOJDNKDF@Debuggee?5status?5sync?5aborted?5be@ 0000000180007870     libclassfloadhk007.obj
 0002:000018b0       ??_C@_0CO@PGPGMHBJ@No?5status?5sync?5occured?5for?5time@ 00000001800078b0     libclassfloadhk007.obj
 0002:000018e0       ??_C@_0CL@DOEBDPKJ@Debuggee?5was?5not?5suspended?5on?5s@ 00000001800078e0     libclassfloadhk007.obj
 0002:00001910       ??_C@_0EA@EEOEJAEN@status?5?$DN?5syncDebuggeeStatus?$CIjni@ 0000000180007910     libclassfloadhk007.obj
 0002:00001950       ??_C@_0BL@JBCFNBMB@nsk_jvmti_resetAgentData?$CI?$CJ@ 0000000180007950     libclassfloadhk007.obj
 0002:00001970       ??_C@_0DN@NNGECJON@jvmti_env?9?$DOSetEventNotification@ 0000000180007970     libclassfloadhk007.obj
 0002:000019b0       ??_C@_0EL@LPBEELIP@s?2test?2hotspot?2jtreg?2vmTestbase@ 00000001800079b0     libclassfloadhk007.obj
 0002:00001a00       ??_C@_0CK@JDAMFDMJ@jvmti?9?$DOSetTag?$CIo?0?5tag?$CJ?5?$DN?$DN?5JVMTI_@ 0000000180007a00     libclassfloadhk007.obj
 0002:00001a30       ??_C@_0CC@DAMNHKNI@Can?8t?5set?5tag?5?$CFli?5for?5object?5?$CFl@ 0000000180007a30     libclassfloadhk007.obj
 0002:00001a58       ??_C@_0DL@HAJPNKEF@jvmti?9?$DOGetObjectHashCode?$CIo?0?5?$CGha@ 0000000180007a58     libclassfloadhk007.obj
 0002:00001a98       ??_C@_0BL@JFPIEOBF@Can?8t?5get?5hash?5object?5?$CFlx?6@ 0000000180007a98     libclassfloadhk007.obj
 0002:00001ab8       ??_C@_0BG@DICPHBKN@setTag?3?5?$CF08x?5?$DM?9?5?$CF?53li@ 0000000180007ab8     libclassfloadhk007.obj
 0002:00001ad0       ??_C@_0DH@FCEEBDMJ@?$CIs?5?$DN?5jni?9?$DOGetStringUTFChars?$CIsIn@ 0000000180007ad0     libclassfloadhk007.obj
 0002:00001b08       ??_C@_0BJ@OKKGHDCN@Can?8t?5get?5string?5at?5?$CF?$CDp?6@ 0000000180007b08     libclassfloadhk007.obj
 0002:00001b28       ??_C@_0BP@EKFLGGFJ@Can?8t?5get?5string?5at?5?$CF?$CDp?3?5null?6@ 0000000180007b28     libclassfloadhk007.obj
 0002:00001b48       ??_C@_06ICODBHCL@?5?1?1?5?$CFs@ 0000000180007b48     libclassfloadhk007.obj
 0002:00001b50       ??_C@_0DB@KGFPLEGO@?$CIr?5?$DN?5jvmti?9?$DOGetTag?$CIo?0?5?$CGtag?$CJ?$CJ?5?$DN?$DN@ 0000000180007b50     libclassfloadhk007.obj
 0002:00001b88       ??_C@_0CO@PDAGBCGJ@Can?8t?5GetTag?5for?5object?5?$CFlx?4?5Re@ 0000000180007b88     libclassfloadhk007.obj
 0002:00001bb8       ??_C@_0CH@HPEODOHC@TEST_BUG?3?5Max?4?5number?5of?5refs?5r@ 0000000180007bb8     libclassfloadhk007.obj
 0002:00001be0       ??_C@_0DI@PHFCABIM@?$CIr?5?$DN?5jvmti?9?$DOGetTag?$CIfrom?0?5?$CGtagFr@ 0000000180007be0     libclassfloadhk007.obj
 0002:00001c18       ??_C@_0DI@MDEGFNKD@TEST_BUG?3?5Can?8t?5GetTag?5for?5obje@ 0000000180007c18     libclassfloadhk007.obj
 0002:00001c50       ??_C@_0DE@MLELJAHM@?$CIr?5?$DN?5jvmti?9?$DOGetTag?$CIto?0?5?$CGtagTo?$CJ?$CJ@ 0000000180007c50     libclassfloadhk007.obj
 0002:00001c88       ??_C@_0BM@KIPKBEMO@Check?5?$CFs?5bytecode?3?50x?$CFp?3?$CFd?6@ 0000000180007c88     libclassfloadhk007.obj
 0002:00001cb0       ??_C@_0GA@BKCPCNEB@s?2test?2hotspot?2jtreg?2vmTestbase@ 0000000180007cb0     libclassfloadhk007.obj
 0002:00001d10       ??_C@_0EG@JHGGAFJI@Unexpected?5null?5pointer?5to?5?$CFs?5b@ 0000000180007d10     libclassfloadhk007.obj
 0002:00001d60       ??_C@_0EB@NFFGOCIE@Unexpected?5zero?5size?5of?5?$CFs?5byte@ 0000000180007d60     libclassfloadhk007.obj
 0002:00001db0       ??_C@_0FL@PLDMGCOM@Unexpected?5size?5of?5?$CFs?5bytecode?5@ 0000000180007db0     libclassfloadhk007.obj
 0002:00001e10       ??_C@_0GK@LBEAAFFJ@Unexpected?5bytes?5in?5?$CFs?5bytecode@ 0000000180007e10     libclassfloadhk007.obj
 0002:00001e80       ??_C@_0DN@DINENAIL@Got?5?$CFs?5bytecode?5is?5not?5equal?5to@ 0000000180007e80     libclassfloadhk007.obj
 0002:00001ec0       ??_C@_0CK@GMIAOFHH@All?5?$CFs?5bytecode?5is?5equal?5to?5exp@ 0000000180007ec0     libclassfloadhk007.obj
 0002:00001ef0       ??_C@_0BH@PMPIFENK@Find?5static?5field?3?5?$CFs?6@ 0000000180007ef0     libclassfloadhk007.obj
 0002:00001f10       ??_C@_0EH@GDANDMKF@?$CIfieldID?5?$DN?5jni?9?$DOGetStaticFieldI@ 0000000180007f10     libclassfloadhk007.obj
 0002:00001f58       ??_C@_0BJ@MIIADDIH@?5?5?4?4?4?5got?5fieldID?3?50x?$CFp?6@ 0000000180007f58     libclassfloadhk007.obj
 0002:00001f78       ??_C@_0DB@LNBEDBAK@Get?5classfile?5bytes?5array?5from?5@ 0000000180007f78     libclassfloadhk007.obj
 0002:00001fb0       ??_C@_0EK@LHJIFLLO@?$CIarray?5?$DN?5?$CIjbyteArray?$CJ?5jni?9?$DOGetS@ 0000000180007fb0     libclassfloadhk007.obj
 0002:00002000       ??_C@_0BO@MCBIMNON@?5?5?4?4?4?5got?5array?5object?3?50x?$CFp?6@ 0000000180008000     libclassfloadhk007.obj
 0002:00002020       ??_C@_0CJ@IMCLCODJ@?$CI?$CKsize?5?$DN?5jni?9?$DOGetArrayLength?$CIar@ 0000000180008020     libclassfloadhk007.obj
 0002:00002050       ??_C@_0CA@DFOMIFBE@?5?5?4?4?4?5got?5array?5size?3?5?$CFd?5bytes?6@ 0000000180008050     libclassfloadhk007.obj
 0002:00002070       ??_C@_0EC@BMGANPNC@?$CIelements?5?$DN?5jni?9?$DOGetByteArrayEl@ 0000000180008070     libclassfloadhk007.obj
 0002:000020b8       ??_C@_0BP@GHIKCANC@?5?5?4?4?4?5got?5elements?5list?3?50x?$CFp?6@ 00000001800080b8     libclassfloadhk007.obj
 0002:000020d8       ??_C@_0BO@INNLGEFF@jvmti?9?$DOAllocate?$CI?$CKsize?0?5bytes?$CJ@ 00000001800080d8     libclassfloadhk007.obj
 0002:000020f8       ??_C@_0CB@GPMKAPNC@?5?5?4?4?4?5created?5bytes?5array?3?50x?$CFp@ 00000001800080f8     libclassfloadhk007.obj
 0002:00002120       ??_C@_0CB@JLCJNBFH@?5?5?4?4?4?5copied?5bytecode?3?5?$CFd?5bytes@ 0000000180008120     libclassfloadhk007.obj
 0002:00002148       ??_C@_0BN@BNPEJKFL@Release?5elements?5list?3?50x?$CFp?6@ 0000000180008148     libclassfloadhk007.obj
 0002:00002168       ??_C@_0DK@LPBJCMNH@jni?9?$DOReleaseByteArrayElements?$CIa@ 0000000180008168     libclassfloadhk007.obj
 0002:000021a8       ??_C@_0BA@MKNEJBDK@?5?5?4?4?4?5released?6@ 00000001800081a8     libclassfloadhk007.obj
 0002:000021b8       ??_C@_0CC@CDBPBOEE@Get?5object?5from?5static?5field?3?5?$CF@ 00000001800081b8     libclassfloadhk007.obj
 0002:000021e0       ??_C@_0DL@FNJHMICH@?$CIobj?5?$DN?5jni?9?$DOGetStaticObjectFiel@ 00000001800081e0     libclassfloadhk007.obj
 0002:00002220       ??_C@_0BI@FNLCMIKO@?5?5?4?4?4?5got?5object?3?50x?$CFp?6@ 0000000180008220     libclassfloadhk007.obj
 0002:00002238       ??_C@_0CH@FJOAJGII@Make?5global?5reference?5to?5object@ 0000000180008238     libclassfloadhk007.obj
 0002:00002260       ??_C@_0CK@GMJMFMJB@?$CIobj?5?$DN?5jni?9?$DONewGlobalRef?$CIobj?$CJ?$CJ?5@ 0000000180008260     libclassfloadhk007.obj
 0002:00002290       ??_C@_0BM@GHFLFCIF@?5?5?4?4?4?5got?5global?5ref?3?50x?$CFp?6@ 0000000180008290     libclassfloadhk007.obj
 0002:000022b0       ??_C@_0BE@CKPNMDMJ@Redefine?5class?3?5?$CFs?6@ 00000001800082b0     libclassfloadhk007.obj
 0002:000022c8       ??_C@_0CF@OBOBAJEI@jvmti?9?$DORedefineClasses?$CI1?0?5?$CGclas@ 00000001800082c8     libclassfloadhk007.obj
 0002:000022f0       ??_C@_0CK@IIFLLALD@?5?5?5?4?4?4?5redefined?5with?5bytecode?3@ 00000001800082f0     libclassfloadhk007.obj
 0002:00002320       ??_C@_0CK@IBLJJBJL@Wait?5for?5debuggee?5to?5load?5origi@ 0000000180008320     libclassfloadhk007.obj
 0002:00002350       ??_C@_0BP@LAIJOMPC@nsk_jvmti_waitForSync?$CItimeout?$CJ@ 0000000180008350     libclassfloadhk007.obj
 0002:00002370       ??_C@_0BL@HCDKGPKD@?$DO?$DO?$DO?5Obtain?5debuggee?5class?6@ 0000000180008370     libclassfloadhk007.obj
 0002:00002390       ??_C@_0CM@GNDDEEM@nsk?1jvmti?1ClassFileLoadHook?1cla@ 0000000180008390     libclassfloadhk007.obj
 0002:000023c0       ??_C@_0BI@ENEOJHP@Find?5debugee?5class?3?5?$CFs?6@ 00000001800083c0     libclassfloadhk007.obj
 0002:000023d8       ??_C@_0DP@MFMMLPOM@?$CIdebugeeClass?5?$DN?5jni?9?$DOFindClass?$CI@ 00000001800083d8     libclassfloadhk007.obj
 0002:00002418       ??_C@_0BJ@DFGCANJI@?5?5?4?4?4?5found?5class?3?50x?$CFp?6@ 0000000180008418     libclassfloadhk007.obj
 0002:00002438       ??_C@_0CA@IJJJOEKD@?$DO?$DO?$DO?5Obtain?5tested?5class?5object?6@ 0000000180008438     libclassfloadhk007.obj
 0002:00002460       ??_C@_0HJ@OOMLALKH@?$CItestedClass?5?$DN?5?$CIjclass?$CJ?5getObje@ 0000000180008460     libclassfloadhk007.obj
 0002:000024e0       ??_C@_0BC@JPHKFLAG@Ljava?1lang?1Class?$DL@ 00000001800084e0     libclassfloadhk007.obj
 0002:000024f8       ??_C@_0M@NBBHFNNO@testedClass@ 00000001800084f8     libclassfloadhk007.obj
 0002:00002508       ??_C@_0BP@BDGPBFBA@?$DO?$DO?$DO?5Obtain?5classloader?5object?6@ 0000000180008508     libclassfloadhk007.obj
 0002:00002530       ??_C@_0GP@ELACKPIG@?$CIclassLoader?5?$DN?5getObject?$CIjvmti?0@ 0000000180008530     libclassfloadhk007.obj
 0002:000025a0       ??_C@_0DJ@PMPPEOPL@Lnsk?1jvmti?1ClassFileLoadHook?1cl@ 00000001800085a0     libclassfloadhk007.obj
 0002:000025e0       ??_C@_0M@GNPGALCO@classLoader@ 00000001800085e0     libclassfloadhk007.obj
 0002:000025f0       ??_C@_0CP@BDBMFEOO@?$DO?$DO?$DO?5Obtain?5redefined?5bytecode?5o@ 00000001800085f0     libclassfloadhk007.obj
 0002:00002620       ??_C@_0HI@FDFFCGFN@getBytecode?$CIjvmti?0?5jni?0?5debugee@ 0000000180008620     libclassfloadhk007.obj
 0002:00002698       ??_C@_02KCBIMKDL@?$FLB@    0000000180008698     libclassfloadhk007.obj
 0002:000026a0       ??_C@_0BA@FDMOBGPB@redefClassBytes@ 00000001800086a0     libclassfloadhk007.obj
 0002:000026b0       ??_C@_0BL@GEMPMCNO@?$DO?$DO?$DO?5Redefine?5tested?5class?6@ 00000001800086b0     libclassfloadhk007.obj
 0002:000026d0       ??_C@_0FG@CLHLABOE@redefineClass?$CIjvmti?0?5testedClas@ 00000001800086d0     libclassfloadhk007.obj
 0002:00002728       ??_C@_0CN@GCGFMFPL@nsk?1jvmti?1ClassFileLoadHook?1cla@ 0000000180008728     libclassfloadhk007.obj
 0002:00002760       ??_C@_0EG@NNNIKMOM@?$DO?$DO?$DO?5Testcase?5?$CD1?3?5Redefine?5class@ 0000000180008760     libclassfloadhk007.obj
 0002:000027a8       ??_C@_0BF@OBFAJONN@CLASS_FILE_LOAD_HOOK@ 00000001800087a8     libclassfloadhk007.obj
 0002:000027c0       ??_C@_0BC@GKPEONMH@Enable?5event?3?5?$CFs?6@ 00000001800087c0     libclassfloadhk007.obj
 0002:000027d8       ??_C@_0DJ@GDOKODHN@nsk_jvmti_enableEvents?$CIJVMTI_EN@ 00000001800087d8     libclassfloadhk007.obj
 0002:00002818       ??_C@_0BF@FDILEKIF@?5?5?4?4?4?5event?5enabled?6@ 0000000180008818     libclassfloadhk007.obj
 0002:00002830       ??_C@_0BD@DHNHPBHK@Disable?5event?3?5?$CFs?6@ 0000000180008830     libclassfloadhk007.obj
 0002:00002848       ??_C@_0DK@BBGCCCAH@nsk_jvmti_enableEvents?$CIJVMTI_DI@ 0000000180008848     libclassfloadhk007.obj
 0002:00002888       ??_C@_0BG@COFELMBN@?5?5?4?4?4?5event?5disabled?6@ 0000000180008888     libclassfloadhk007.obj
 0002:000028a0       ??_C@_0CB@NPDGNJKL@Check?5if?5event?5was?5received?3?5?$CFs@ 00000001800088a0     libclassfloadhk007.obj
 0002:000028d0       ??_C@_0GL@MHHLBGFJ@Unexpected?5number?5of?5?$CFs?5events?5@ 00000001800088d0     libclassfloadhk007.obj
 0002:00002940       ??_C@_0BL@KAEJJGL@?5?5?4?4?4?5received?3?5?$CFd?5events?6@ 0000000180008940     libclassfloadhk007.obj
 0002:00002960       ??_C@_0BF@MNKEFEOE@?$DO?$DO?$DO?5Clean?5used?5data?6@ 0000000180008960     libclassfloadhk007.obj
 0002:00002978       ??_C@_0DF@HFEDKLDB@Delete?5global?5reference?5to?5clas@ 0000000180008978     libclassfloadhk007.obj
 0002:000029b0       ??_C@_0DG@BJFGMMDE@Delete?5global?5reference?5to?5test@ 00000001800089b0     libclassfloadhk007.obj
 0002:000029e8       ??_C@_0CL@NCGHDDJM@Deallocate?5redefined?5bytecode?5a@ 00000001800089e8     libclassfloadhk007.obj
 0002:00002a18       ??_C@_0CD@IIHFKBFE@jvmti?9?$DODeallocate?$CIredefClassByt@ 0000000180008a18     libclassfloadhk007.obj
 0002:00002a40       ??_C@_0BH@HPEOJMHL@Let?5debugee?5to?5finish?6@ 0000000180008a40     libclassfloadhk007.obj
 0002:00002a58       ??_C@_0BH@LECMGIIA@nsk_jvmti_resumeSync?$CI?$CJ@ 0000000180008a58     libclassfloadhk007.obj
 0002:00002a70       ??_C@_0FG@EBADLIEI@?5?5?$DMCLASS_FILE_LOAD_HOOK?$DO?3?5name?3@ 0000000180008a70     libclassfloadhk007.obj
 0002:00002ac8       ??_C@_0DE@BFHJPBEF@SUCCESS?$CB?5CLASS_FILE_LOAD_HOOK?5f@ 0000000180008ac8     libclassfloadhk007.obj
 0002:00002b00       ??_C@_0BJ@GOBDGGIC@Check?5classloader?3?50x?$CFp?6@ 0000000180008b00     libclassfloadhk007.obj
 0002:00002b20       ??_C@_0DL@PGLFLHFL@Unexpected?5null?5classloader?5in?5@ 0000000180008b20     libclassfloadhk007.obj
 0002:00002b60       ??_C@_0GH@NCFLCHPM@Unexpected?5classloader?5in?5CLASS@ 0000000180008b60     libclassfloadhk007.obj
 0002:00002bc8       ??_C@_0CD@HCKIEBCH@Check?5class_being_redefined?3?50x@ 0000000180008bc8     libclassfloadhk007.obj
 0002:00002bf0       ??_C@_0EF@BEHBAOAJ@Unexpected?5null?5class_being_red@ 0000000180008bf0     libclassfloadhk007.obj
 0002:00002c40       ??_C@_0HB@IIFOBKNJ@Unexpected?5class_being_redefine@ 0000000180008c40     libclassfloadhk007.obj
 0002:00002cb8       ??_C@_09KLOJBFOH@redefined@ 0000000180008cb8     libclassfloadhk007.obj
 0002:00002cc8       ??_C@_0CA@MNKGCBCG@nsk_jvmti_parseOptions?$CIoptions?$CJ@ 0000000180008cc8     libclassfloadhk007.obj
 0002:00002ce8       ??_C@_0DN@MIAMNFPH@?$CIjvmti?5?$DN?5nsk_jvmti_createJVMTIE@ 0000000180008ce8     libclassfloadhk007.obj
 0002:00002d28       ??_C@_0DL@CAHEFBHA@can_generate_eraly_class_hook_e@ 0000000180008d28     libclassfloadhk007.obj
 0002:00002d68       ??_C@_0BP@CGFOKBDM@Add?5required?5capabilities?3?5?$CFs?6@ 0000000180008d68     libclassfloadhk007.obj
 0002:00002d88       ??_C@_0BO@DBKDIPGD@jvmti?9?$DOAddCapabilities?$CI?$CGcaps?$CJ@ 0000000180008d88     libclassfloadhk007.obj
 0002:00002da8       ??_C@_0N@GCANCHC@?5?5?4?4?4?5added?6@ 0000000180008da8     libclassfloadhk007.obj
 0002:00002db8       ??_C@_0BM@DNBHNNGB@Set?5callback?5for?5event?3?5?$CFs?6@ 0000000180008db8     libclassfloadhk007.obj
 0002:00002dd8       ??_C@_0CL@LMFMDJFG@jvmti?9?$DOSetEventCallbacks?$CI?$CGcallb@ 0000000180008dd8     libclassfloadhk007.obj
 0002:00002e08       ??_C@_0L@HIMFBJJO@?5?5?4?4?4?5set?6@ 0000000180008e08     libclassfloadhk007.obj
 0002:00002e18       ??_C@_0CL@PIACJIPK@nsk_jvmti_setAgentProc?$CIagentPro@ 0000000180008e18     libclassfloadhk007.obj
 0002:00002e60       ??_C@_1EC@JIJBPKFM@?$AAa?$AAp?$AAi?$AA?9?$AAm?$AAs?$AA?9?$AAw?$AAi?$AAn?$AA?9?$AAc?$AAo?$AAr?$AAe@ 0000000180008e60     MSVCRT:thread_safe_statics.obj
 0002:00002ea8       ??_C@_1BK@MGMFAEKH@?$AAk?$AAe?$AAr?$AAn?$AAe?$AAl?$AA3?$AA2?$AA?4?$AAd?$AAl?$AAl@ 0000000180008ea8     MSVCRT:thread_safe_statics.obj
 0002:00002ec8       ??_C@_0BJ@JEBJOJFJ@SleepConditionVariableCS@ 0000000180008ec8     MSVCRT:thread_safe_statics.obj
 0002:00002ee8       ??_C@_0BJ@PGPPEPCC@WakeAllConditionVariable@ 0000000180008ee8     MSVCRT:thread_safe_statics.obj
 0002:00002f08       _pDefaultRawDllMain        0000000180008f08     MSVCRT:dll_dllmain.obj
 0002:00002f08       _pRawDllMain               0000000180008f08     MSVCRT:dll_dllmain.obj
 0002:00002f10       __xmm@ffffffffffffffffffffffffffffffff 0000000180008f10     MSVCRT:utility.obj
 0002:00002f20       _load_config_used          0000000180008f20     MSVCRT:loadcfg.obj
 0002:00003100       _tls_used                  0000000180009100     MSVCRT:tlssup.obj
 0002:00003128       __volatile_metadata        0000000180009128     <linker-defined>
 0002:00003558       __rtc_iaa                  0000000180009558     MSVCRT:initsect.obj
 0002:00003560       __rtc_izz                  0000000180009560     MSVCRT:initsect.obj
 0002:00003568       __rtc_taa                  0000000180009568     MSVCRT:initsect.obj
 0002:00003570       __rtc_tzz                  0000000180009570     MSVCRT:initsect.obj
 0002:00003578       _tls_start                 0000000180009578     MSVCRT:tlssup.obj
 0002:0000357c       _Init_thread_epoch         000000018000957c     MSVCRT:thread_safe_statics.obj
 0002:00003580       _tls_end                   0000000180009580     MSVCRT:tlssup.obj
 0002:00003cd8       __IMPORT_DESCRIPTOR_KERNEL32 0000000180009cd8     kernel32:KERNEL32.dll
 0002:00003cec       __IMPORT_DESCRIPTOR_VCRUNTIME140 0000000180009cec     vcruntime:VCRUNTIME140.dll
 0002:00003d00       __IMPORT_DESCRIPTOR_api-ms-win-crt-heap-l1-1-0 0000000180009d00     ucrt:api-ms-win-crt-heap-l1-1-0.dll
 0002:00003d14       __IMPORT_DESCRIPTOR_api-ms-win-crt-runtime-l1-1-0 0000000180009d14     ucrt:api-ms-win-crt-runtime-l1-1-0.dll
 0002:00003d28       __IMPORT_DESCRIPTOR_api-ms-win-crt-convert-l1-1-0 0000000180009d28     ucrt:api-ms-win-crt-convert-l1-1-0.dll
 0002:00003d3c       __IMPORT_DESCRIPTOR_api-ms-win-crt-stdio-l1-1-0 0000000180009d3c     ucrt:api-ms-win-crt-stdio-l1-1-0.dll
 0002:00003d50       __IMPORT_DESCRIPTOR_api-ms-win-crt-string-l1-1-0 0000000180009d50     ucrt:api-ms-win-crt-string-l1-1-0.dll
 0002:00003d64       __NULL_IMPORT_DESCRIPTOR   0000000180009d64     kernel32:KERNEL32.dll
 0003:00000030       _Init_global_epoch         000000018000b030     MSVCRT:thread_safe_statics.obj
 0003:00000040       __security_cookie          000000018000b040     MSVCRT:gs_cookie.obj
 0003:00000048       __security_cookie_complement 000000018000b048     MSVCRT:gs_cookie.obj
 0003:00000050       __scrt_native_dllmain_reason 000000018000b050     MSVCRT:utility.obj
 0003:00000058       __isa_available            000000018000b058     MSVCRT:cpu_disp.obj
 0003:0000005c       __isa_enabled              000000018000b05c     MSVCRT:cpu_disp.obj
 0003:00000060       __memset_fast_string_threshold 000000018000b060     MSVCRT:cpu_disp.obj
 0003:00000068       __memset_nt_threshold      000000018000b068     MSVCRT:cpu_disp.obj
 0003:00000070       __scrt_ucrt_dll_is_in_use  000000018000b070     MSVCRT:ucrt_stubs.obj
 0003:00000080       g_wrongHeapCallbacks       000000018000b080     libclassfloadhk007.obj
 0003:00000100       g_szTagInfo                000000018000b100     libclassfloadhk007.obj
 0003:00002040       g_tagFlags                 000000018000d040     libclassfloadhk007.obj
 0003:00002428       g_refsToVerifyCnt          000000018000d428     libclassfloadhk007.obj
 0003:0000242c       g_fakeUserData             000000018000d42c     libclassfloadhk007.obj
 0003:00002430       g_tagVisitCount            000000018000d430     libclassfloadhk007.obj
 0003:000033d0       g_refsToVerify             000000018000e3d0     libclassfloadhk007.obj
 0003:0001aad0       g_userDataError            0000000180025ad0     libclassfloadhk007.obj
 0003:0001ac90       ?_OptionsStorage@?1??__local_stdio_printf_options@@9@4_KA 0000000180025c90     libclassfloadhk007.obj
 0003:0001b258       _tls_index                 0000000180026258     MSVCRT:tlssup.obj
 0003:0001b260       __scrt_current_native_startup_state 0000000180026260     MSVCRT:utility.obj
 0003:0001b268       __scrt_native_startup_lock 0000000180026268     MSVCRT:utility.obj
 0003:0001b2a8       __scrt_debugger_hook_flag  00000001800262a8     MSVCRT:utility_desktop.obj
 0003:0001b2b0       ?__type_info_root_node@@3U__type_info_node@@A 00000001800262b0     MSVCRT:tncleanup.obj
 0003:0001b2c0       ?_OptionsStorage@?1??__local_stdio_scanf_options@@9@4_KA 00000001800262c0     MSVCRT:default_local_stdio_options.obj
 0003:0001b2c8       __favor                    00000001800262c8     MSVCRT:cpu_disp.obj
 0003:0001b2d0       __dyn_tls_init_callback    00000001800262d0     <common>

 entry point at        0001:00003f10

 Static symbols

 0000:fffd7000       .debug$S                   0000000180000000     classfloadhk007.exp
 0000:fffd7000       .debug$S                   0000000180000000     vcruntime:VCRUNTIME140.dll
 0000:fffd7000       .debug$S                   0000000180000000     vcruntime:VCRUNTIME140.dll
 0000:fffd7000       .debug$S                   0000000180000000     vcruntime:VCRUNTIME140.dll
 0000:fffd7000       .debug$S                   0000000180000000     vcruntime:VCRUNTIME140.dll
 0000:fffd7000       .debug$S                   0000000180000000     vcruntime:VCRUNTIME140.dll
 0000:fffd7000       .debug$S                   0000000180000000     vcruntime:VCRUNTIME140.dll
 0000:fffd7000       .debug$S                   0000000180000000     vcruntime:VCRUNTIME140.dll
 0000:fffd7000       .debug$S                   0000000180000000     ucrt:api-ms-win-crt-convert-l1-1-0.dll
 0000:fffd7000       .debug$S                   0000000180000000     ucrt:api-ms-win-crt-heap-l1-1-0.dll
 0000:fffd7000       .debug$S                   0000000180000000     ucrt:api-ms-win-crt-heap-l1-1-0.dll
 0000:fffd7000       .debug$S                   0000000180000000     ucrt:api-ms-win-crt-heap-l1-1-0.dll
 0000:fffd7000       .debug$S                   0000000180000000     ucrt:api-ms-win-crt-heap-l1-1-0.dll
 0000:fffd7000       .debug$S                   0000000180000000     ucrt:api-ms-win-crt-runtime-l1-1-0.dll
 0000:fffd7000       .debug$S                   0000000180000000     ucrt:api-ms-win-crt-runtime-l1-1-0.dll
 0000:fffd7000       .debug$S                   0000000180000000     ucrt:api-ms-win-crt-runtime-l1-1-0.dll
 0000:fffd7000       .debug$S                   0000000180000000     ucrt:api-ms-win-crt-runtime-l1-1-0.dll
 0000:fffd7000       .debug$S                   0000000180000000     ucrt:api-ms-win-crt-runtime-l1-1-0.dll
 0000:fffd7000       .debug$S                   0000000180000000     ucrt:api-ms-win-crt-runtime-l1-1-0.dll
 0000:fffd7000       .debug$S                   0000000180000000     ucrt:api-ms-win-crt-runtime-l1-1-0.dll
 0000:fffd7000       .debug$S                   0000000180000000     ucrt:api-ms-win-crt-runtime-l1-1-0.dll
 0000:fffd7000       .debug$S                   0000000180000000     ucrt:api-ms-win-crt-runtime-l1-1-0.dll
 0000:fffd7000       .debug$S                   0000000180000000     ucrt:api-ms-win-crt-runtime-l1-1-0.dll
 0000:fffd7000       .debug$S                   0000000180000000     ucrt:api-ms-win-crt-runtime-l1-1-0.dll
 0000:fffd7000       .debug$S                   0000000180000000     ucrt:api-ms-win-crt-runtime-l1-1-0.dll
 0000:fffd7000       .debug$S                   0000000180000000     ucrt:api-ms-win-crt-runtime-l1-1-0.dll
 0000:fffd7000       .debug$S                   0000000180000000     ucrt:api-ms-win-crt-runtime-l1-1-0.dll
 0000:fffd7000       .debug$S                   0000000180000000     ucrt:api-ms-win-crt-runtime-l1-1-0.dll
 0000:fffd7000       .debug$S                   0000000180000000     ucrt:api-ms-win-crt-runtime-l1-1-0.dll
 0000:fffd7000       .debug$S                   0000000180000000     ucrt:api-ms-win-crt-stdio-l1-1-0.dll
 0000:fffd7000       .debug$S                   0000000180000000     ucrt:api-ms-win-crt-stdio-l1-1-0.dll
 0000:fffd7000       .debug$S                   0000000180000000     ucrt:api-ms-win-crt-stdio-l1-1-0.dll
 0000:fffd7000       .debug$S                   0000000180000000     ucrt:api-ms-win-crt-stdio-l1-1-0.dll
 0000:fffd7000       .debug$S                   0000000180000000     ucrt:api-ms-win-crt-stdio-l1-1-0.dll
 0000:fffd7000       .debug$S                   0000000180000000     ucrt:api-ms-win-crt-stdio-l1-1-0.dll
 0000:fffd7000       .debug$S                   0000000180000000     ucrt:api-ms-win-crt-stdio-l1-1-0.dll
 0000:fffd7000       .debug$S                   0000000180000000     ucrt:api-ms-win-crt-stdio-l1-1-0.dll
 0000:fffd7000       .debug$S                   0000000180000000     ucrt:api-ms-win-crt-stdio-l1-1-0.dll
 0000:fffd7000       .debug$S                   0000000180000000     ucrt:api-ms-win-crt-stdio-l1-1-0.dll
 0000:fffd7000       .debug$S                   0000000180000000     ucrt:api-ms-win-crt-string-l1-1-0.dll
 0000:fffd7000       .debug$S                   0000000180000000     ucrt:api-ms-win-crt-string-l1-1-0.dll
 0000:fffd7000       .debug$S                   0000000180000000     ucrt:api-ms-win-crt-string-l1-1-0.dll
 0000:fffd7000       .debug$S                   0000000180000000     ucrt:api-ms-win-crt-string-l1-1-0.dll
 0000:fffd7000       .debug$S                   0000000180000000     ucrt:api-ms-win-crt-string-l1-1-0.dll
 0000:fffd7000       .debug$S                   0000000180000000     ucrt:api-ms-win-crt-string-l1-1-0.dll
 0000:fffd7000       .debug$S                   0000000180000000     ucrt:api-ms-win-crt-string-l1-1-0.dll
 0000:fffd7000       .debug$S                   0000000180000000     ucrt:api-ms-win-crt-string-l1-1-0.dll
 0000:fffd7000       .debug$S                   0000000180000000     kernel32:KERNEL32.dll
 0000:fffd7000       .debug$S                   0000000180000000     kernel32:KERNEL32.dll
 0000:fffd7000       .debug$S                   0000000180000000     kernel32:KERNEL32.dll
 0000:fffd7000       .debug$S                   0000000180000000     kernel32:KERNEL32.dll
 0000:fffd7000       .debug$S                   0000000180000000     kernel32:KERNEL32.dll
 0000:fffd7000       .debug$S                   0000000180000000     kernel32:KERNEL32.dll
 0000:fffd7000       .debug$S                   0000000180000000     kernel32:KERNEL32.dll
 0000:fffd7000       .debug$S                   0000000180000000     kernel32:KERNEL32.dll
 0000:fffd7000       .debug$S                   0000000180000000     kernel32:KERNEL32.dll
 0000:fffd7000       .debug$S                   0000000180000000     kernel32:KERNEL32.dll
 0000:fffd7000       .debug$S                   0000000180000000     kernel32:KERNEL32.dll
 0000:fffd7000       .debug$S                   0000000180000000     kernel32:KERNEL32.dll
 0000:fffd7000       .debug$S                   0000000180000000     kernel32:KERNEL32.dll
 0000:fffd7000       .debug$S                   0000000180000000     kernel32:KERNEL32.dll
 0000:fffd7000       .debug$S                   0000000180000000     kernel32:KERNEL32.dll
 0000:fffd7000       .debug$S                   0000000180000000     kernel32:KERNEL32.dll
 0000:fffd7000       .debug$S                   0000000180000000     kernel32:KERNEL32.dll
 0000:fffd7000       .debug$S                   0000000180000000     kernel32:KERNEL32.dll
 0000:fffd7000       .debug$S                   0000000180000000     kernel32:KERNEL32.dll
 0000:fffd7000       .debug$S                   0000000180000000     kernel32:KERNEL32.dll
 0000:fffd7000       .debug$S                   0000000180000000     kernel32:KERNEL32.dll
 0000:fffd7000       .debug$S                   0000000180000000     kernel32:KERNEL32.dll
 0000:fffd7000       .debug$S                   0000000180000000     kernel32:KERNEL32.dll
 0000:fffd7000       .debug$S                   0000000180000000     kernel32:KERNEL32.dll
 0000:fffd7000       .debug$S                   0000000180000000     kernel32:KERNEL32.dll
 0000:fffd7000       .debug$S                   0000000180000000     kernel32:KERNEL32.dll
 0000:fffd7000       .debug$S                   0000000180000000     kernel32:KERNEL32.dll
 0000:fffd7000       .debug$S                   0000000180000000     kernel32:KERNEL32.dll
 0001:00000f04       addRefToVerify             0000000180001f04 f   libclassfloadhk007.obj
 0001:00000f78       agentProc                  0000000180001f78 f   libclassfloadhk007.obj
 0001:00001634       agentThreadWrapper         0000000180002634 f   libclassfloadhk007.obj
 0001:00001788       callbackClassFileLoadHook  0000000180002788 f   libclassfloadhk007.obj
 0001:00001998       checkBytecode              0000000180002998 f   libclassfloadhk007.obj
 0001:00001b48       check_option               0000000180002b48 f   libclassfloadhk007.obj
 0001:00001d90       file_basename              0000000180002d90 f   libclassfloadhk007.obj
 0001:00001e04       getBytecode                0000000180002e04 f   libclassfloadhk007.obj
 0001:00002224       getObject                  0000000180003224 f   libclassfloadhk007.obj
 0001:000031ac       redefineClass              00000001800041ac f   libclassfloadhk007.obj
 0001:00003300       startAgentThreadWrapper    0000000180004300 f   libclassfloadhk007.obj
 0001:0000362c       syncDebuggeeStatus         000000018000462c f   libclassfloadhk007.obj
 0001:00003964       capture_current_context    0000000180004964 f   MSVCRT:gs_report.obj
 0001:000039d4       capture_previous_context   00000001800049d4 f   MSVCRT:gs_report.obj
 0001:00003a48       ?__scrt_initialize_thread_safe_statics@@YAHXZ 0000000180004a48 f   MSVCRT:thread_safe_statics.obj
 0001:00003b18       ?__scrt_uninitialize_thread_safe_statics@@YAXXZ 0000000180004b18 f   MSVCRT:thread_safe_statics.obj
 0001:00003bc0       $$000000                   0000000180004bc0     MSVCRT:amdsecgs.obj
 0001:00003bf0       ?dllmain_crt_dispatch@@YAHQEAUHINSTANCE__@@KQEAX@Z 0000000180004bf0 f   MSVCRT:dll_dllmain.obj
 0001:00003c40       ?dllmain_crt_process_attach@@YAHQEAUHINSTANCE__@@QEAX@Z 0000000180004c40 f   MSVCRT:dll_dllmain.obj
 0001:00003d58       ?dllmain_crt_process_detach@@YAH_N@Z 0000000180004d58 f   MSVCRT:dll_dllmain.obj
 0001:00003ddc       ?dllmain_dispatch@@YAHQEAUHINSTANCE__@@KQEAX@Z 0000000180004ddc f   MSVCRT:dll_dllmain.obj
 0001:00004800       $$000000                   0000000180005800     MSVCRT:guard_dispatch.obj
 0001:00004820       $$000000                   0000000180005820     MSVCRT:guard_xfg_dispatch.obj
 0001:00004836       ?fin$0@?0??dllmain_crt_process_attach@@YAHQEAUHINSTANCE__@@QEAX@Z@4HA 0000000180005836 f   MSVCRT:dll_dllmain.obj
 0001:0000484d       ?fin$0@?0??dllmain_crt_process_detach@@YAH_N@Z@4HA 000000018000584d f   MSVCRT:dll_dllmain.obj
 0001:00004866       ?fin$1@?0??dllmain_crt_process_detach@@YAH_N@Z@4HA 0000000180005866 f   MSVCRT:dll_dllmain.obj
 0001:0000487a       ?filt$0@?0??dllmain_dispatch@@YAHQEAUHINSTANCE__@@KQEAX@Z@4HA 000000018000587a f   MSVCRT:dll_dllmain.obj
 0001:000048b0       __scrt_is_nonwritable_in_current_image$filt$0 00000001800058b0 f   MSVCRT:utility.obj
 0002:00000228       ?__scrt_initialize_tss_var@@3P6AHXZEA 0000000180006228     MSVCRT:thread_safe_statics.obj
 0002:00000350       ?opcLengths@@3QBEB         0000000180006350     libclassfloadhk007.obj
 0002:00002e48       GS_ExceptionPointers       0000000180008e48     MSVCRT:gs_report.obj
 0002:00003588       $unwind$fprintf            0000000180009588     libclassfloadhk007.obj
 0002:00003594       $unwind$printf             0000000180009594     libclassfloadhk007.obj
 0002:000035a0       $unwind$snprintf           00000001800095a0     libclassfloadhk007.obj
 0002:000035b0       $unwind$?NewObject@JNIEnv_@@QEAAPEAV_jobject@@PEAV_jclass@@PEAU_jmethodID@@ZZ 00000001800095b0     libclassfloadhk007.obj
 0002:000035b0       $unwind$nsk_lcomplain      00000001800095b0     libclassfloadhk007.obj
 0002:000035b0       $unwind$nsk_ldisplay       00000001800095b0     libclassfloadhk007.obj
 0002:000035b8       $unwind$nsk_lvdisplay      00000001800095b8     libclassfloadhk007.obj
 0002:000035b8       $unwind$_RTC_Initialize    00000001800095b8     MSVCRT:initsect.obj
 0002:000035b8       $unwind$_RTC_Terminate     00000001800095b8     MSVCRT:initsect.obj
 0002:000035b8       $unwind$?__scrt_initialize_thread_safe_statics@@YAHXZ 00000001800095b8     MSVCRT:thread_safe_statics.obj
 0002:000035c4       $unwind$nsk_complain       00000001800095c4     libclassfloadhk007.obj
 0002:000035c4       $unwind$nsk_printf         00000001800095c4     libclassfloadhk007.obj
 0002:000035cc       $unwind$nsk_lvcomplain     00000001800095cc     libclassfloadhk007.obj
 0002:000035e4       $unwind$nsk_ltrace         00000001800095e4     libclassfloadhk007.obj
 0002:000035e4       $unwind$__report_gsfailure 00000001800095e4     MSVCRT:gs_report.obj
 0002:000035ec       $unwind$nsk_lvtrace        00000001800095ec     libclassfloadhk007.obj
 0002:000035ec       $unwind$__raise_securityfailure 00000001800095ec     MSVCRT:gs_report.obj
 0002:000035ec       $unwind$__scrt_initialize_crt 00000001800095ec     MSVCRT:utility.obj
 0002:000035ec       $unwind$__scrt_initialize_onexit_tables 00000001800095ec     MSVCRT:utility.obj
 0002:000035ec       $unwind$__scrt_release_startup_lock 00000001800095ec     MSVCRT:utility.obj
 0002:000035ec       $unwind$__scrt_uninitialize_crt 00000001800095ec     MSVCRT:utility.obj
 0002:000035ec       $unwind$_onexit            00000001800095ec     MSVCRT:utility.obj
 0002:000035f4       $unwind$nsk_lverify        00000001800095f4     libclassfloadhk007.obj
 0002:00003604       $unwind$nsk_vprintf        0000000180009604     libclassfloadhk007.obj
 0002:00003614       $unwind$nsk_printHexBytes  0000000180009614     libclassfloadhk007.obj
 0002:00003638       $unwind$?nsk_jni_lverify@@YAHHPEAUJNIEnv_@@HQEBDH1ZZ 0000000180009638     libclassfloadhk007.obj
 0002:0000364c       $unwind$?nsk_jni_check_exception@@YAHPEAUJNIEnv_@@QEBDH@Z 000000018000964c     libclassfloadhk007.obj
 0002:00003668       $unwind$nsk_jvmti_parseOptions 0000000180009668     libclassfloadhk007.obj
 0002:00003684       $unwind$nsk_jvmti_createJVMTIEnv 0000000180009684     libclassfloadhk007.obj
 0002:00003698       $unwind$check_option       0000000180009698     libclassfloadhk007.obj
 0002:00003698       $unwind$nsk_jvmti_waitForSync 0000000180009698     libclassfloadhk007.obj
 0002:00003698       $unwind$_DllMainCRTStartup 0000000180009698     MSVCRT:dll_dllmain.obj
 0002:000036a8       $unwind$Java_nsk_jvmti_unit_FollowReferences_FollowRefObjects_resetTags 00000001800096a8     libclassfloadhk007.obj
 0002:000036a8       $unwind$addRefToVerify     00000001800096a8     libclassfloadhk007.obj
 0002:000036a8       $unwind$nsk_jvmti_resetAgentData 00000001800096a8     libclassfloadhk007.obj
 0002:000036a8       $unwind$nsk_jvmti_resumeSync 00000001800096a8     libclassfloadhk007.obj
 0002:000036a8       $unwind$__scrt_initialize_default_local_stdio_options 00000001800096a8     MSVCRT:default_local_stdio_options.obj
 0002:000036a8       $unwind$?dllmain_crt_dispatch@@YAHQEAUHINSTANCE__@@KQEAX@Z 00000001800096a8     MSVCRT:dll_dllmain.obj
 0002:000036a8       $unwind$DllMain            00000001800096a8     MSVCRT:dll_dllmain_stub.obj
 0002:000036a8       $unwind$__report_rangecheckfailure 00000001800096a8     MSVCRT:gs_report.obj
 0002:000036a8       $unwind$__GSHandlerCheck   00000001800096a8     MSVCRT:gshandler.obj
 0002:000036a8       $unwind$?__scrt_uninitialize_thread_safe_statics@@YAXXZ 00000001800096a8     MSVCRT:thread_safe_statics.obj
 0002:000036a8       $unwind$__scrt_acquire_startup_lock 00000001800096a8     MSVCRT:utility.obj
 0002:000036a8       $unwind$__scrt_dllmain_after_initialize_c 00000001800096a8     MSVCRT:utility.obj
 0002:000036a8       $unwind$__scrt_dllmain_before_initialize_c 00000001800096a8     MSVCRT:utility.obj
 0002:000036a8       $unwind$__scrt_dllmain_crt_thread_attach 00000001800096a8     MSVCRT:utility.obj
 0002:000036a8       $unwind$__scrt_dllmain_crt_thread_detach 00000001800096a8     MSVCRT:utility.obj
 0002:000036a8       $unwind$__scrt_dllmain_uninitialize_c 00000001800096a8     MSVCRT:utility.obj
 0002:000036a8       $unwind$__scrt_dllmain_uninitialize_critical 00000001800096a8     MSVCRT:utility.obj
 0002:000036a8       $unwind$atexit             00000001800096a8     MSVCRT:utility.obj
 0002:000036b0       $unwind$nsk_jvmti_enableEvents 00000001800096b0     libclassfloadhk007.obj
 0002:000036c8       $unwind$nsk_jvmti_lverify  00000001800096c8     libclassfloadhk007.obj
 0002:000036dc       $unwind$exitOnError        00000001800096dc     libclassfloadhk007.obj
 0002:000036ec       $unwind$Java_nsk_share_jvmti_ArgumentHandler_getAgentOptionsString 00000001800096ec     libclassfloadhk007.obj
 0002:00003700       $unwind$Java_nsk_jvmti_unit_FollowReferences_FollowRefObjects_getTag 0000000180009700     libclassfloadhk007.obj
 0002:00003700       $unwind$Java_nsk_share_jvmti_DebugeeClass_checkStatus 0000000180009700     libclassfloadhk007.obj
 0002:00003700       $unwind$agentThreadWrapper 0000000180009700     libclassfloadhk007.obj
 0002:00003710       $unwind$agentProc          0000000180009710     libclassfloadhk007.obj
 0002:00003710       $unwind$startAgentThreadWrapper 0000000180009710     libclassfloadhk007.obj
 0002:0000372c       $unwind$syncDebuggeeStatus 000000018000972c     libclassfloadhk007.obj
 0002:0000372c       $unwind$__scrt_dllmain_exception_filter 000000018000972c     MSVCRT:utility.obj
 0002:00003740       $unwind$Java_nsk_share_jvmti_DebugeeClass_resetAgentData 0000000180009740     libclassfloadhk007.obj
 0002:00003748       $unwind$MA_checkStatus     0000000180009748     libclassfloadhk007.obj
 0002:0000375c       $unwind$Java_nsk_jvmti_unit_FollowReferences_FollowRefObjects_setTag 000000018000975c     libclassfloadhk007.obj
 0002:00003774       $unwind$Java_nsk_jvmti_unit_FollowReferences_FollowRefObjects_addRefToVerify 0000000180009774     libclassfloadhk007.obj
 0002:00003774       $unwind$callbackClassFileLoadHook 0000000180009774     libclassfloadhk007.obj
 0002:00003790       $unwind$Agent_Initialize   0000000180009790     libclassfloadhk007.obj
 0002:000037b0       $unwind$checkBytecode      00000001800097b0     libclassfloadhk007.obj
 0002:000037c8       $unwind$getBytecode        00000001800097c8     libclassfloadhk007.obj
 0002:000037e4       $unwind$getObject          00000001800097e4     libclassfloadhk007.obj
 0002:00003800       $unwind$redefineClass      0000000180009800     libclassfloadhk007.obj
 0002:00003814       $unwind$__report_securityfailure 0000000180009814     MSVCRT:gs_report.obj
 0002:0000381c       $unwind$capture_current_context 000000018000981c     MSVCRT:gs_report.obj
 0002:00003828       $unwind$capture_previous_context 0000000180009828     MSVCRT:gs_report.obj
 0002:00003834       $unwind$__GSHandlerCheckCommon 0000000180009834     MSVCRT:gshandler.obj
 0002:00003840       $xdatasym                  0000000180009840     MSVCRT:amdsecgs.obj
 0002:00003844       $unwind$?dllmain_crt_process_attach@@YAHQEAUHINSTANCE__@@QEAX@Z 0000000180009844     MSVCRT:dll_dllmain.obj
 0002:00003880       $unwind$?fin$0@?0??dllmain_crt_process_attach@@YAHQEAUHINSTANCE__@@QEAX@Z@4HA 0000000180009880     MSVCRT:dll_dllmain.obj
 0002:00003880       $unwind$?fin$0@?0??dllmain_crt_process_detach@@YAH_N@Z@4HA 0000000180009880     MSVCRT:dll_dllmain.obj
 0002:00003880       $unwind$?fin$1@?0??dllmain_crt_process_detach@@YAH_N@Z@4HA 0000000180009880     MSVCRT:dll_dllmain.obj
 0002:00003888       $unwind$?dllmain_crt_process_detach@@YAH_N@Z 0000000180009888     MSVCRT:dll_dllmain.obj
 0002:000038dc       $unwind$?dllmain_dispatch@@YAHQEAUHINSTANCE__@@KQEAX@Z 00000001800098dc     MSVCRT:dll_dllmain.obj
 0002:00003904       $unwind$?filt$0@?0??dllmain_dispatch@@YAHQEAUHINSTANCE__@@KQEAX@Z@4HA 0000000180009904     MSVCRT:dll_dllmain.obj
 0002:0000390c       $unwind$__scrt_is_nonwritable_in_current_image 000000018000990c     MSVCRT:utility.obj
 0002:0000392c       $unwind$__scrt_is_nonwritable_in_current_image$filt$0 000000018000992c     MSVCRT:utility.obj
 0002:00003934       $unwind$__scrt_fastfail    0000000180009934     MSVCRT:utility_desktop.obj
 0002:00003944       $unwind$__security_init_cookie 0000000180009944     MSVCRT:gs_support.obj
 0002:00003950       $unwind$__isa_available_init 0000000180009950     MSVCRT:cpu_disp.obj
 0002:00003960       $xdatasym                  0000000180009960     MSVCRT:guard_dispatch.obj
 0002:00003968       $xdatasym                  0000000180009968     MSVCRT:guard_xfg_dispatch.obj
 0002:00003970       .edata                     0000000180009970     classfloadhk007.exp
 0002:00003998       rgpv                       0000000180009998     classfloadhk007.exp
 0002:000039d0       rgszName                   00000001800099d0     classfloadhk007.exp
 0002:00003a08       rgwOrd                     0000000180009a08     classfloadhk007.exp
 0002:00003a24       szName                     0000000180009a24     classfloadhk007.exp
 0002:00003a38       $N00001                    0000000180009a38     classfloadhk007.exp
 0002:00003a47       $N00002                    0000000180009a47     classfloadhk007.exp
 0002:00003a54       $N00003                    0000000180009a54     classfloadhk007.exp
 0002:00003a99       $N00004                    0000000180009a99     classfloadhk007.exp
 0002:00003ad6       $N00005                    0000000180009ad6     classfloadhk007.exp
 0002:00003b1e       $N00006                    0000000180009b1e     classfloadhk007.exp
 0002:00003b5e       $N00007                    0000000180009b5e     classfloadhk007.exp
 0002:00003b9b       $N00008                    0000000180009b9b     classfloadhk007.exp
 0002:00003bd6       $N00009                    0000000180009bd6     classfloadhk007.exp
 0002:00003c04       $N00010                    0000000180009c04     classfloadhk007.exp
 0002:00003c35       $N00011                    0000000180009c35     classfloadhk007.exp
 0002:00003c64       $N00012                    0000000180009c64     classfloadhk007.exp
 0002:00003c93       $N00013                    0000000180009c93     classfloadhk007.exp
 0002:00003cc8       $N00014                    0000000180009cc8     classfloadhk007.exp
 0002:0000413a       .idata$6                   000000018000a13a     kernel32:KERNEL32.dll
 0002:0000419e       .idata$6                   000000018000a19e     vcruntime:VCRUNTIME140.dll
 0002:00004344       .idata$6                   000000018000a344     ucrt:api-ms-win-crt-heap-l1-1-0.dll
 0002:00004364       .idata$6                   000000018000a364     ucrt:api-ms-win-crt-runtime-l1-1-0.dll
 0002:00004386       .idata$6                   000000018000a386     ucrt:api-ms-win-crt-convert-l1-1-0.dll
 0002:000043a8       .idata$6                   000000018000a3a8     ucrt:api-ms-win-crt-stdio-l1-1-0.dll
 0002:000043c8       .idata$6                   000000018000a3c8     ucrt:api-ms-win-crt-string-l1-1-0.dll
 0003:00000000       ?codeAttributeName@@3PEBDEB 000000018000b000     libclassfloadhk007.obj
 0003:00000008       ?lineNumberAttributeName@@3PEBDEB 000000018000b008     libclassfloadhk007.obj
 0003:00000010       ?localVarAttributeName@@3PEBDEB 000000018000b010     libclassfloadhk007.obj
 0003:00000018       ?localVarTypeAttributeName@@3PEBDEB 000000018000b018     libclassfloadhk007.obj
 0003:00000020       ?stackMapAttributeName@@3PEBDEB 000000018000b020     libclassfloadhk007.obj
 0003:00000028       ?callBytes@@3PAEA          000000018000b028     libclassfloadhk007.obj
 0003:0000002c       ?allocBytes@@3PAEA         000000018000b02c     libclassfloadhk007.obj
 0003:0001aad4       redefineAttempted          0000000180025ad4     libclassfloadhk007.obj
 0003:0001aad8       nsk_context                0000000180025ad8     libclassfloadhk007.obj
 0003:0001aae4       redefineSucceed            0000000180025ae4     libclassfloadhk007.obj
 0003:0001aae8       agentFailed                0000000180025ae8     libclassfloadhk007.obj
 0003:0001aaec       currentAgentStatus         0000000180025aec     libclassfloadhk007.obj
 0003:0001aaf0       context                    0000000180025af0     libclassfloadhk007.obj
 0003:0001aba8       agentThread                0000000180025ba8     libclassfloadhk007.obj
 0003:0001abb0       agentThreadProc            0000000180025bb0     libclassfloadhk007.obj
 0003:0001abb8       agentThreadArg             0000000180025bb8     libclassfloadhk007.obj
 0003:0001abc0       agent_data                 0000000180025bc0     libclassfloadhk007.obj
 0003:0001abd0       jvmti_env                  0000000180025bd0     libclassfloadhk007.obj
 0003:0001abd8       jvm                        0000000180025bd8     libclassfloadhk007.obj
 0003:0001abe0       jni_env                    0000000180025be0     libclassfloadhk007.obj
 0003:0001abe8       checkStatus_func           0000000180025be8     libclassfloadhk007.obj
 0003:0001abf0       ?codeAttributeIndex@@3GA   0000000180025bf0     libclassfloadhk007.obj
 0003:0001abf4       ?lineNumberAttributeIndex@@3GA 0000000180025bf4     libclassfloadhk007.obj
 0003:0001abf8       ?localVarAttributeIndex@@3GA 0000000180025bf8     libclassfloadhk007.obj
 0003:0001abfc       ?localVarTypeAttributeIndex@@3GA 0000000180025bfc     libclassfloadhk007.obj
 0003:0001ac00       ?stackMapAttributeIndex@@3GA 0000000180025c00     libclassfloadhk007.obj
 0003:0001ac04       ?stackFrameOffset@@3GA     0000000180025c04     libclassfloadhk007.obj
 0003:0001ac08       ?mode@@3HA                 0000000180025c08     libclassfloadhk007.obj
 0003:0001ac0c       ?constantPoolSize@@3GA     0000000180025c0c     libclassfloadhk007.obj
 0003:0001ac10       ?orig@@3PEBEEB             0000000180025c10     libclassfloadhk007.obj
 0003:0001ac18       ?gen@@3PEAEEA              0000000180025c18     libclassfloadhk007.obj
 0003:0001ac20       ?inputPos@@3PEAEEA         0000000180025c20     libclassfloadhk007.obj
 0003:0001ac28       ?endPos@@3PEBEEB           0000000180025c28     libclassfloadhk007.obj
 0003:0001ac30       ?genPos@@3PEAEEA           0000000180025c30     libclassfloadhk007.obj
 0003:0001ac38       ?markPos@@3PEAEEA          0000000180025c38     libclassfloadhk007.obj
 0003:0001ac40       ?constantPool@@3PEAPEADEA  0000000180025c40     libclassfloadhk007.obj
 0003:0001ac48       ?constantPoolCount@@3GA    0000000180025c48     libclassfloadhk007.obj
 0003:0001ac4c       ?zeroBytes@@3PAEA          0000000180025c4c     libclassfloadhk007.obj
 0003:0001ac50       ?codeLength@@3IA           0000000180025c50     libclassfloadhk007.obj
 0003:0001ac54       redefClassSize             0000000180025c54     libclassfloadhk007.obj
 0003:0001ac58       ?map@@3PEAIEA              0000000180025c58     libclassfloadhk007.obj
 0003:0001ac60       ?widening@@3PEACEA         0000000180025c60     libclassfloadhk007.obj
 0003:0001ac68       timeout                    0000000180025c68     libclassfloadhk007.obj
 0003:0001ac70       classLoader                0000000180025c70     libclassfloadhk007.obj
 0003:0001ac78       testedClass                0000000180025c78     libclassfloadhk007.obj
 0003:0001ac80       redefClassBytes            0000000180025c80     libclassfloadhk007.obj
 0003:0001ac88       eventsCount                0000000180025c88     libclassfloadhk007.obj
 0003:0001aca0       GS_ExceptionRecord         0000000180025ca0     MSVCRT:gs_report.obj
 0003:0001ad40       GS_ContextRecord           0000000180025d40     MSVCRT:gs_report.obj
 0003:0001b210       ?g_tss_cv@@3U_RTL_CONDITION_VARIABLE@@A 0000000180026210     MSVCRT:thread_safe_statics.obj
 0003:0001b218       ?g_tss_event@@3PEAXEA      0000000180026218     MSVCRT:thread_safe_statics.obj
 0003:0001b220       ?g_tss_mutex@@3U_RTL_CRITICAL_SECTION@@A 0000000180026220     MSVCRT:thread_safe_statics.obj
 0003:0001b248       ?g_sleep_condition_variable_cs@@3P6AHPEAU_RTL_CONDITION_VARIABLE@@PEAU_RTL_CRITICAL_SECTION@@K@ZEA 0000000180026248     MSVCRT:thread_safe_statics.obj
 0003:0001b250       ?g_wake_all_condition_variable@@3P6AXPEAU_RTL_CONDITION_VARIABLE@@@ZEA 0000000180026250     MSVCRT:thread_safe_statics.obj
 0003:0001b25c       ?__proc_attached@@3HA      000000018002625c     MSVCRT:dll_dllmain.obj
 0003:0001b270       ?is_initialized_as_dll@@3_NA 0000000180026270     MSVCRT:utility.obj
 0003:0001b271       ?module_local_atexit_table_initialized@@3_NA 0000000180026271     MSVCRT:utility.obj
 0003:0001b278       ?module_local_atexit_table@@3U_onexit_table_t@@A 0000000180026278     MSVCRT:utility.obj
 0003:0001b290       ?module_local_at_quick_exit_table@@3U_onexit_table_t@@A 0000000180026290     MSVCRT:utility.obj
